:020000040800F2
:10500000D0170020D5500008D1950008B58C0008B5
:105010000000000000000000000000000000000090
:1050200000000000000000000000000055A1000882
:105030000000000000000000C99D0008E5A2000873
:10504000E7500008E7500008E7500008E750000864
:10505000E7500008A9670008E75000081568000835
:1050600000000000E750000829640008E75000082D
:10507000E75000089D91000800000000E75000087C
:1050800000000000E75000080000000000000000E1
:10509000E750000800000000E7500008E750000853
:1050A000E7500008E7500008E75000085DAD000831
:1050B000E7500008E7500008000000000000000072
:1050C0000348854600F01AFD0048004739C3000830
:1050D000D01700200448804704480047FEE7FEE759
:1050E000FEE7FEE7FEE7FEE781A30008C1500008E7
:1050F00030B50B46014600202022012409E00D4670
:10510000D5409D4205D31D469540491B25469540F7
:1051100040191546521E002DF1DC30BD70B500243B
:105120002546002801DA01244042002901DA012540
:105130004942FFF7DDFFAC4200D04042002C00D0D6
:10514000494270BDF0B51FB40646002082B0054646
:105150004024019100901BE0019922460F46304601
:1051600000F0CAFB049A059B801A994110D310469F
:105170001946224600F0B0FB361A8F4101972246AD
:1051800001200021009F00F0A7FB38184D4100903E
:105190002046641E0028DFDC019B00982946324629
:1051A00007B0F0BD03460B439B0703D009E008C9D5
:1051B000121F08C0042AFAD203E00B780370401CC7
:1051C000491C521EF9D27047D2B201E00270401C55
:1051D000491EFBD270470022F6E710B513460A4677
:1051E00004461946FFF7F0FF204610BD30B50446CF
:1051F0000020034600E05B1C934203D2E05CCD5CE0
:10520000401BF8D030BDF8B502464A40D40F4200EA
:105210004B0052085B089A4202D2024608461146E9
:105220004A0023D0C30D4A00DDB2120EAD1A202D64
:1052300035DA49020126490AF6058A19002C00D000
:10524000524220214F1B1146B9402A411018C20D6D
:105250009A4221D0002C17D0012D08DCDA05801AE3
:10526000D20F8019D207DBB200F072FBF8BDDA056D
:10527000801A012340001B06C01880185A4280186B
:10528000CA0F1043490007E04908C2071143DA0575
:10529000801A80194008801800F052FBF8BD6100A8
:1052A0000122511A001BF7E70122D2075140AAE759
:1052B0000122D2075040A6E770B502464A40D50FFA
:1052C00040004A00ED0740085208002814D0002A88
:1052D00012D0C40DD30D41020120C0055202490A6B
:1052E000520AE41A091812187D34914201D3641C41
:1052F00000E04900002C01DA002070BD002391423B
:1053000001D3891A0343400849000028F7D1002936
:105310000AD0914202D10121C90705E0914201D290
:10532000012101E00121C943E005C018401900F046
:1053300007FB70BDF0B507460846584087B0C00F60
:10534000049048000E46590040084908BC1A88419C
:1053500005D2384631461E4617460B4602465800CF
:10536000400810434CD0300D039040055900400DCB
:10537000490D0590401A0290402872DA1803012165
:10538000000B09050843019004980092002805D0FD
:1053900001995242002088410092019002984021D8
:1053A0000A1A0199009800F097FA05460C466B46D8
:1053B00007CB00F0B2FAC0197141039A0E0D002319
:1053C000D71756401A467A40164344D0049A002A0A
:1053D0002DD0029A012A039A15DC1205C01A9141B8
:1053E00001263605001C7141D20F059ED20700939D
:1053F000019202962A46234600F0F0FA07B0F0BD6B
:1054000038463146FAE71605224A0F46B218C01A46
:10541000B74101210905001C4F4100187F41114689
:1054200018187941E20F10436D19644113E0E20747
:105430006D0815436408C2071443039A0126120538
:10544000C01A91413605001C7141CE074008304317
:105450004908C01851412A46234600F0B2FACDE768
:10546000FFE7049801224000C117121A00238B4164
:1054700004983146C417381AA141EEE730B401242C
:10548000E407634030BC55E730B40124E4076140D1
:1054900030BC4FE70000E0FFF0B51FB488B00B99B7
:1054A0000998002448400999C00F4900490809910A
:1054B000C0070B990090490049080B910999089879
:1054C000A64608431CD00B990A98084318D009989F
:1054D00001244000420D4800410D099824050003B5
:1054E000000B204309900B980003000B20430B9006
:1054F00050181C494018002201901446104605E03F
:10550000002001460DB0F0BD032801DA034600E09B
:1055100003239C46C11A0AAE0AE05F0008ADED5BAA
:105520004F00F75B7D430027AA187C41491C5B1E96
:105530006145F2DD410004AB5A522104120C0A43CA
:10554000240C401C0828DFDB01980290009970466B
:1055500001910090059B049A0799069800F03EFA85
:10556000D0E700000DFCFFFFF0B50C465C4085B0B5
:10557000E40FE40703944C000026640859009446A5
:10558000490802460296224321D062460A431ED0B1
:105590006200570D4A000E032303550D01240246F5
:1055A0002C492405781B1B0B360B4018234326433C
:1055B000614600901C46501AB44103D30098401C29
:1055C000009002E0921800985B41002803DA002066
:1055D000014605B0F0BD00200121090507468646B9
:1055E00011E064461D46141BB54106D36546521BA7
:1055F000B341744607430C43A646CD07400849080B
:10560000284392185B4105460D43EAD110461843E2
:1056100013D06046194650407140084306D060469A
:10562000101AB34106D20122002306E00022012312
:10563000DB0702E00122D2435310009874460105B3
:10564000381C6141029C039D0019694100F0B9F9C1
:10565000BFE70000FD03000070B54B005B0803438B
:105660000BD04B005C0D002633466542B341D41786
:10567000AD1AA34102DB0020014670BD12053018AF
:10568000514170BDC217C10F504010B54018CA0734
:105690009623002100F05CF910BD10B5002296237E
:1056A000114600F055F910BD0EB5C217C10F50409C
:1056B000CA0740180021054B0293019200910A4647
:1056C0000B4600F08BF903B000BD0000330400006E
:1056D0000EB505490291002100910A460B46019141
:1056E00000F07CF903B000BD330400003EB5CA17DA
:1056F000CB0F002450405140C0186141DA07054BE0
:105700000293019200942246234600F067F903B009
:1057100030BD000033040000410040020122400A75
:10572000D205090E80187F2901DA002070479629DA
:1057300003DC9622511AC84070479639884070475A
:1057400070B5CD0F4A0009030123090B1B0519434E
:105750000B4BED070024520D9A4201DA002070BD78
:10576000074B34339A4203DC9A1A00F0C5F802E082
:105770000449511888402C43F1D0404270BD0000CC
:10578000FF030000CDFBFFFF4A0009030123090BC3
:105790001B051943094B10B5520D9A4201DA00203E
:1057A00010BD064B34339A4203DC9A1A00F0A4F879
:1057B00010BD03495118884010BD0000FF030000D0
:1057C000CDFBFFFF70B5CD0F4A0009030123090B84
:1057D0001B0519430D4BED070024520D9A4202DAC6
:1057E0000020014670BD094B34339A4203DC9A1AFB
:1057F00000F082F803E0064BD21800F06DF82C435D
:10580000F0D0002240428A41114670BDFF030000E3
:10581000CDFBFFFFC20FD207400040080BD0C10DE7
:105820000723DB01C91840020905400A1143C208D9
:1058300040071143704700200146704710B500290A
:1058400004DB0124E40740428C412146002B04DBA9
:105850001C460123DB075242A3418B4200D1824206
:1058600010BD000010B5002904DB0124E40740420C
:105870008C412146002B04DB1C460123DB075242EE
:10588000A341994200D1904210BD0000CB0FDB072D
:10589000490010B5490802460A4307D00A0D0724FB
:1058A0000903E401090B121B002A01DC002010BDD2
:1058B000C900440F0C43C100E018D205801800F065
:1058C0003FF810BD0122D207002800DB101A002982
:1058D00000DB511A8142704710B5202A04DB0146D3
:1058E000203A9140002010BD914020239C1A03468D
:1058F000E3401943904010BD10B5202A04DB084650
:10590000203AD040002110BD0B46D340D040202487
:10591000A21A91400843194610BD10B5202A06DB93
:10592000CB170846203A1041C1170B4306E00B463F
:105930001341D0402024A21A91400843194610BDBB
:10594000002904DA401C490001D14008400070479A
:1059500070B40024050C05D11024000402D10029E4
:1059600021D01124050E01D100020834050F01D108
:105970000001241D850F01D18000A41C002801DB3B
:105980004000641C002908D020252E1B0D46F54040
:10599000A14000D001212943084301061B1B000A36
:1059A000DB1D02D5002070BC7047DB05181880187D
:1059B0000029F8DA401C4900F5D170BC40084000CD
:1059C000704710B5002B08DA0024401C6141921882
:1059D0005B411A4301D14008400010BDF0B51FB42F
:1059E00082B005460C0003D0084605F08BFA02E0B1
:1059F00005F088FA20300246009021462846FFF73D
:105A00006BFF049B059A04460F4618431143084355
:105A100014D0184610431BD0009840210A1A18468B
:105A20000599FFF769FF05460E46009A0599049807
:105A3000FFF752FF084305D0012004E02046394615
:105A400007B0F0BD0020C11705430E432C43374378
:105A500000990E986305401A7905E40A00220C4368
:105A6000FD0A0A3002D500200146E9E701051019B8
:105A700069410C9C0D9D00196941FFF7A2FFDFE70A
:105A8000F8B50546480040080C46284304D060009D
:105A9000184A400D904201DD2846F8BD15493539B8
:105AA000884210DC88420BDB290D200308432903C0
:105AB000014305D0E00F1049C00741180020F8BD90
:105AC00000200146F8BD161A4020821B28462146B8
:105AD000FFF702FF07460091284621463246FFF7AE
:105AE0000BFF3A46009BFFF76CFF3246FFF7F4FED0
:105AF000F8BD0000330400000000F03F064C012513
:105B0000064E05E0E36807CC2B430C3C9847103465
:105B1000B442F7D3FFF7D8FAE8CA000808CB000868
:105B200070B58C180578401C6B075B0F01D10378AA
:105B3000401C2A1106D10278401C03E006780E7042
:105B4000401C491C5B1EF9D12B0705D40023521EB3
:105B50000DD40B70491CFAE70378401CCB1A921C39
:105B600003E01D780D70491C5B1C521EF9D5A14243
:105B7000D8D3002070BD000038B50446064805495A
:105B80000068FFF7B5FA604300E0401E009000286F
:105B9000FBD138BD40420F005C020020F8B504463E
:105BA000006881688907890F012902D10168C90746
:105BB00022D18168114A10261140012500290ED1F9
:105BC0008168294381600120FFF7D6FF01F042FD83
:105BD00007460CE001F03EFDC01B0A2807D9606DA6
:105BE00030436065A06D2843A0650120F8BD2068A2
:105BF0000068C043C007EDD10020F8BD1700008049
:105C000010B5012006F01CFC0A4C1328A0700AD025
:105C1000E01C03F02BFAE078A070332806D0064988
:105C20000020C88710BD06F043FC10BD03F0F0F95A
:105C300010BD0000000000203C040020F8B5002149
:105C4000664805F0C7FF00210F2005F00BFF644CEC
:105C5000606240047ED50122920300210F2006F0ED
:105C60008AF80021102005F0FDFEC1B2217061709C
:105C700000225C4805F064FF5A4922464B78937332
:105C8000481C8978D1730179217440796074554D2D
:105C9000554B2A781B789A4279D16A7A062A76D1AE
:105CA000EA78A2712A79E271EA792272AA7A62729A
:105CB0002174607429460B3152004C480091FFF763
:105CC00071FA607A42004948511928300B31FFF7C8
:105CD00069FA607A80004019C17A2175007B60758D
:105CE000208A00F085FBE082A189002201268842FB
:105CF00009D13E4FE1824B005037208AF852491CAF
:105D0000A181A67000E0A2703848E18AB430425404
:105D100037480088FFF7C1FC07463648C188608ACB
:105D2000FFF7E6F90846FFF7B8FC3946FFF7C4FA73
:105D3000FFF770FD06F0D0FCFFF7A8FDFFF7ECFCC5
:105D4000C1B22D4A01205054607AA17A884208D904
:105D5000A07200E02AE04200244800992838FFF7AA
:105D600021FA26490026E778607A0A6812E01D4980
:105D700073005D18EB7A69460B702B7B4B700988BA
:105D8000914205D10027304600F03CF804E00CE0D9
:105D9000761CF6B28642EAD3E770607A86420AD170
:105DA0000120E070304600F02DF804E0144A002194
:105DB0000F2005F0E0FF05F003FD114A00210F2040
:105DC00005F0D9FF0121054805F004FF002005F08A
:105DD0002DFF002005F0CDFEF8BD000000D02324EB
:105DE00040010020200A00200D020020740B00203A
:105DF000180200203C040020240D00203402002062
:105E0000F8D02724F0B5FF4A8BB00546FE49FF4C79
:105E10000B78D37549781176217CD176617C117726
:105E200006F043F8FF229132F94B6A43D21813046B
:105E30006166DA17206618184A411106000A0843FD
:105E4000A06205F0C0FE607AFF21401B91314843FB
:105E5000FF309B3005F0D0FEEE4805F0E7FEA0785D
:105E600000280BD0E08AEC4A8100EC484250081828
:105E7000E44A018811844088508408E0E08A810067
:105E8000E6480918DF480A88028449884184E44FBB
:105E9000DC48397816300170072141720021C17445
:105EA0000A460146182005F091FF0021182005F050
:105EB0009FFF032005F0F0FE0006000ED94E207172
:105EC0003AD0401C2071A08C400414D4D64A002142
:105ED0000F2005F050FF002005F04BFE00210F20A1
:105EE00005F0C0FD3042606202D160790028F5D033
:105EF000A08C40047ED58122D20100210F2005F024
:105F00003AFF0021102005F0ADFD4106BD48490EC5
:105F100021700022803805F013FEBA4EE078803EF2
:105F2000002814D00222B849701CFFF75FF900283E
:105F30000DD001200BB0F0BD00210F2005F092FD27
:105F400030426062BFD160790028F5D0BBE7707A3B
:105F50000828EFD1AD4902221031701DFFF746F934
:105F60000028E7D1A7483978803800788842E1D105
:105F700000273E4603A805F0F4FD042003A93A0ECD
:105F8000360216433A020F5C1743401EF7D52765C9
:105F9000666505F08AFFE165A0659C4999482C314A
:105FA000763805F04BFF9748A900803808189749C4
:105FB0001630303105F042FF9449924834316E3842
:105FC00005F03CFF206EA0630790256DE563A66D8C
:105FD0002664206B0290E16A401AFFF779FBE166C4
:105FE000A0660746701B0591FFF772FB616720678B
:105FF000039100E046E10490616B0298081AFFF7F4
:1060000067FBE1670646A06707980191281AFFF72A
:106010005FFB7E4D803503C5009007913846083DF3
:10602000039B049A0599FFF785F93246019BFFF718
:1060300081F9079B009AFFF77DF909910890304696
:10604000079B009A0199FFF727FA06460091384608
:10605000039B049A0599FFF71FFA3246009BFFF74E
:106060000DFA099B089AFFF77FFAFFF7ABFBE9608F
:10607000A860FFF73BFB6D4A6D4BFFF70DFA13224B
:10608000696112066B4B2861FFF706FAE961A861A6
:10609000FFF7FCFB68494A780B780146184605F083
:1060A000B7FBEB69AA69FFF7EFF969620022634B5E
:1060B0002862FFF7F1F9E962A862614805F006FD80
:1060C0005F4803F01FF8A86AE96A06460D46FFF725
:1060D000DDFB5C4908605C490C20085E0A214843EE
:1060E000FFF7E2FA32462B46FFF724F90E46054643
:1060F000FFF726FB6064607A617880000F30884289
:106100000CD11420205E0A214843FFF7CDFA2A461D
:106110003346FFF7B9F9FFF713FB60644848E58A97
:106120000026963846554948676C494938188842D0
:1061300000D3FFE64248AC0010300059381A01D4B1
:10614000024600E042423E4B4249643B8A4202DA48
:1061500001225A5500E05E55002800DA404288428C
:1061600004DB37483238415D03297BD93A480A219C
:1061700006803846FEF7D2FF2449284A8864304911
:106180002F4B32394E55105110331F51C833014631
:10619000002F00DC31481851314E55203070AA20B4
:1061A00070700120B0701120184DF070A879307116
:1061B00030462B7C43716B7C837103461248002967
:1061C0000778DF714078187201DC244810512448A8
:1061D000A11804220930FEF7E5FFE87970730B4C33
:1061E000287AB0738034616B206BFFF7CDFAF073BF
:1061F000E16BA06BFFF7C8FA30741121B01C00F0FE
:10620000E9F830E0A00A002034020020400100201C
:106210009E020000CC100000FFFF01005C0C00207B
:106220000D02002000D0272400902724FA48CE3BFE
:106230001835B13D19DDB1412801002000408F40E3
:10624000EC0D0020340100203C0400209F8601005A
:106250001F0B20001027000090000020FFFF02000D
:10626000900600200BE06946088009480978C1744F
:10627000694649780175152104F08AFD5AE6491CE2
:10628000415557E6034A00210F2005F074FD51E601
:106290009006002000902724F0B5434D89B00024DB
:1062A00042496700085D424A0028D05370D0401E22
:1062B0000855A60010469C3005968059FFF7F4F962
:1062C0000022D2433B4BFFF7E7F8FFF7DFFA3649EE
:1062D0008039C86701903648296870308059401A63
:1062E000FFF7F6F969622862069104903048304958
:1062F0004430183180598959401AFFF7E9F9E962A9
:10630000A86202900E467F20C0050199FEF7CCFFDF
:10631000FFF780FA3346029AFFF7BEF8069B049A0D
:10632000FFF7B2F80022D243FFF796F9224A234B37
:10633000FFF7B2F8132269631206214B2863FFF7B7
:10634000ABF8E96100221F4BA861FFF78BFA24D25A
:1063500000221D4BE969A869FFF770FA1DD21448A5
:10636000C830C05FFFF7A0F906460F460022174B62
:10637000E969A869FFF790F832463B46FEF7DAFF75
:10638000FFF7DEF9094A0599303A505005E0FFE77A
:106390000648A2000E4930388150641C0B2C00DAEC
:1063A0007EE709B0F0BD0000F00000205407002097
:1063B00078080020FFFF0FBEFA48CE3B1835B13DEC
:1063C00019DDB14100408FC0006AF840000059401B
:1063D000FFFF010010B500231A4603E0845CE318B8
:1063E0009BB2521C8A42F9D3D84380B210BD000040
:1063F000F1B500240A4E0B4D09E06000811902221C
:106400006846FEF7F3FE002804D0641CA4B2A889F5
:106410008442F2D302490020643108552046F8BD79
:10642000C40B00204001002010B5034800F0B6FE68
:10643000024800F0B3FE10BD7013002028130020A6
:1064400030B5446C1C252C400125A540046C6560CA
:10645000046863608368102B036803D09960006848
:10646000C26030BD9A600068C16030BDF0B58BB0CD
:1064700000200790884E0A2005F0BEFB7D204001D9
:1064800005F0D4FB854C0025206C401C206484481A
:106490000990FF38813808900021814861710B30E4
:1064A000226CC270120A027281740A2141727D4903
:1064B00009788172E18C017345707B4909980A78EB
:1064C00002744978417476491C2000220B3105F092
:1064D0007DFC60790621484300211C3005F088FCD2
:1064E000022005F0D9FB714F00210F2005F0BAFA08
:1064F00038426064F8D0606C411C16D040047DD5F1
:106500008122D20100210F2005F035FC002110204E
:1065100005F0A8FA4106490E0022654805F010FB77
:10652000634F787A022802D09FE004F049FD0222EE
:106530005D49781DFEF75AFE00287DD105F0C8FCA4
:10654000564A803203C205F09DFC544A8032D16025
:10655000906002900798039100281AD101205449B5
:10656000079054482839CB8E0380098F524AFF3157
:10657000C33189B2A18491420BD952428918A184B6
:106580005B1C4D4A99B20B320180914201D300212C
:106590000180434B69000B330898CA18017A0A91AD
:1065A000D174407A04904249107528394A8E684661
:1065B0008280898EC1800422791C581CFEF7F2FD6E
:1065C0000198B04205DA064669460A9808750498AB
:1065D000487533480C210B304172304F4B220299E1
:1065E0008037D20403980023891858410206080A0C
:1065F0001043019005F0E7FA019800E04AE04008F6
:106600004000010E00027961386125480CCF153039
:10661000083F05F020FC2248FB681930BA6805F0F5
:106620001AFC1F487B691D303A6905F014FC1C49AF
:1066300000220B31192000E017E005F0C7FB002114
:10664000192005F0D5FB012005F026FB0006000E01
:10665000207305D100210F2005F004FA0006F9D5BA
:10666000802200210F2005F086FB6D1CEDB20A2D63
:1066700000D211E7084886420AD0002E08D0002038
:106680006073022020706846808A208500F0D4F96B
:106690000BB0F0BD094AE4E7FFFF010070000020E5
:1066A000A50700201E0200203402002000D027246D
:1066B0002C06002040020020E70300000090272461
:1066C00010B5104C6078002807D0002060700821B9
:1066D0000D4802F03DF80D4807E0012060700821E8
:1066E000094802F035F87D20C00000F027FE08219F
:1066F000054802F06BF806486178C18006F03AF868
:1067000010BD0000080200209C110020B80B000002
:106710007C0400201449012048720A4602205E329F
:10672000507203203C3A507204200E3A50720F48C7
:106730000D4B0078087022310870203108770C4921
:106740005A1C087858714978997123331871597116
:10675000203318775977107551751A461E32107507
:106760005175107651767047040500200D02002007
:106770003402002010B503F0C3FC202003F0A8FD74
:10678000012005F0A9F8002003F0A2FD044804F060
:10679000FBFE044805F040FA002005F075FA10BD34
:1067A000280100208380000070B503F09FFD0520C4
:1067B0000121000700F03AFF0025144C002800D00A
:1067C00065600221124800F031FF002816D1012037
:1067D00020707F21A068C905884204DB00F010F911
:1067E0006080A56009E000F00BF96188401A80B272
:1067F0003338F92801D2FFF763FF6560012000F00C
:106800004DFE022000F04AFE70BD00004402002050
:106810000004005010B5FF20013000F03FFE10BD15
:106820007047000010B5084900224A6107494B68CB
:106830004C1523434B604B68082423434B60C0092D
:10684000C001026010BD0000B8130020002002400B
:106850007FB500250C460646039500F0E9FDE009EA
:10686000029003A901960095684600F079FD002882
:1068700004D000F0B1FD002004B070BD00F0ACFD0C
:106880000120F9E710B5002302E0C45CCC545B1C86
:106890009342FAD310BD000010B5214A002190693F
:1068A000C305204804D5416902231943416191156C
:1068B00093699B0505D54369012423434361630222
:1068C000194393695B0505D5436908242343436154
:1068D000E301194393691B0505D543690424234348
:1068E00043616302194393699B0405D543691024EE
:1068F000234343616302194393699B0304D54469AD
:1069000020231C43446119439369DB0305D5436984
:10691000402423434361A0020143916110BD000064
:1069200000200240B813002070B5054600F092FE2A
:106930000646184C0AE0681C08D0002D04D000F070
:1069400089FE801BA84201D9032070BDA069C00741
:10695000F1D1A069800701D50220A061A069C0051E
:1069600011D4A06980050ED4A06940050BD4A0699C
:10697000000508D4A069800405D4A069800302D46E
:10698000A069C00303D5FFF787FF012070BD002079
:1069900070BD000000200240F8B5174600260546ED
:1069A0000C4600F045FD09E029460220226800F06F
:1069B00021FD002804D1241D2D1D361DBE42F3D318
:1069C00000F00AFDBE4201D20020F8BD0120F8BD52
:1069D00010B5084902460020054B497905E04400FE
:1069E0001C5B944203D0401CC0B28842F7D310BD58
:1069F000C20600207000002010B500F01CFE10BD83
:106A000010B5094801F03CF880B2FEF761FE074A74
:106A1000074BFEF741FD0022064BFEF7A5FDFEF7F2
:106A2000B3FE80B210BD000014110020F853E3A59E
:106A30009B843E4000408F4070B50024204603F008
:106A40005BF947494748A200641CE4B281500C2C12
:106A5000F9D3464944480A7A0275497A417544494E
:106A60000A780276497841763F49152013314872F9
:106A70000A2005F0C1F87D20400105F0D7F83A4919
:106A8000002213310C2005F0A1F900210C2005F0A3
:106A9000AFF9384800F0F4FF344C0125203C608504
:106AA000AD0309E0334800F0EBFF80B26085218F31
:106AB000FF392D39884206DB218F80B28842F1D31D
:106AC00049198842EED8022005F0E6F8002003F0CC
:106AD00013F9294D00210F2004F0C4FF28426064FF
:106AE000F8D0606C411C38D0400435D58122D201E9
:106AF00000210F2005F03FF90021102004F0B2FF23
:106B000041061948490E0022C73005F019F8164D04
:106B1000C735687A15281FD102221549681DFEF76E
:106B200065FB002818D11148AE7C66710422691CEF
:106B30003C30FEF737FB29461331084672000D46FC
:106B40008330FEF72FFB60792946420005484A381A
:106B5000FEF728FB0320207070BD04F031FA00001E
:106B6000FFFF0100240700206505002090000020A1
:106B7000340200201411002000D0272410B508484A
:106B800000F096FA0A21064800F032FA044800F0B4
:106B90001DF9800503D5024800F01AF980B210BD36
:106BA000B8100020F8B52F4D00220121284600F032
:106BB0004AFDFFF7E3FFFEF770FD2B4E3146FEF76F
:106BC0007BFB2A4C0122A0601146284600F03BFDC9
:106BD0002749A068002588423EDB2078254F002801
:106BE00015D02570FFF7CAFFFEF757FD3146FEF7B7
:106BF00063FBA060FEF70EFE00223B46FEF73EFC64
:106C000000221D4BFEF748FCFEF740FE6060A068C6
:106C1000FEF700FE00223B46FEF730FC174A184BF9
:106C2000FEF73AFC06460F466068FEF7F3FD134A8E
:106C3000144B5242FEF730FC32463B46FEF77AFBDD
:106C4000FEF724FE10496060884201DD616004E0C7
:106C5000FF21C905C84200D365606068FEF75CFD8E
:106C6000C0B2F8BD0004005000401B4448000020A2
:106C70000000604000000C4000E0644033333333D8
:106C800033B33040CCCCEC3F0000C842F8B50546E9
:106C900004464035287C0026012808D001202874AD
:106CA000206881688907890F01290ED101E002203F
:106CB000F8BD0168C90708D0606D202108436065F0
:106CC0000126002028743046F8BD616DFF22013294
:106CD0009143022211436165C1688907890F0091C0
:106CE000C16889088900C1602068816892071143E2
:106CF000816000F0AFFC07460EE000F0ABFCC01B6B
:106D00000A2809D9606D0221884310210843606573
:106D1000002028740120F8BD206880680028ECDB82
:106D20002068C168009A1143C160606D80088000CE
:106D3000401C6065C5E70000F8B506460D464036C4
:106D4000317C01290DD00121317401688A68520714
:106D500009D5416D20221143416500203074012086
:106D6000F8BD0220F8BD174B6A68D80547109A4253
:106D7000154C8A6A2B6812D05B035B0B1A438A623C
:106D80002968490305D5A1680143A1600A20FEF7DF
:106D9000F3FE2868800312D5A06838430EE05B0339
:106DA0005B0B9A438A622968490302D5A168814333
:106DB000A1602868800302D5A068B843A0600020C5
:106DC0003074F8BD0110000000270140406D70478D
:106DD0000068006C7047000070B5040006D0606D5C
:106DE000264600254036002802D006E0012070BD6E
:106DF000A5653574204600F0D3F8606DC00603D455
:106E000021688868400705D5606D102108436065DA
:106E10003574EBE7606DFF2201329043022210438C
:106E2000606588688207920F5B48012A02D10A6870
:106E3000D2072BD1032362689B079A4205D05B429D
:106E40009A4202D05B009A4209D10A6992009208E4
:106E50000A6121680A6963681A430A610CE00A69D9
:106E6000920092080A6181680F2292049143816026
:106E700081686268114381602168CA6818239A4357
:106E8000CA602168CA68A3681A43CA60816801227F
:106E90005206914381608168A28E5206114381603F
:106EA00020688168C90004D4816801221207114357
:106EB00081602068C168394A1140C1602069E16879
:106EC000022825D000200143204620300278037B91
:106ED00052035B001A431143226B1143A2699203D0
:106EE0001143E269D20311432268D3681943D16088
:106EF000616A0A46FF3AC23A05D0A26A1143226883
:106F0000D3681943D16042780121012A02D00BE0F5
:106F10000420D8E70078002823D0606D2022104399
:106F20006065A06D0843A065E06B012820681FD054
:106F30000169C90703D00169490849000161206856
:106F40004169C908C900416120684169A26B1143C8
:106F50004161A565606D80088000401C606500206F
:106F600070BD2068C26801231B041A43C260DBE7BE
:106F70000269FF239B009A43026120680269236C27
:106F8000A66C1A43636C33431A430261206802699A
:106F90000A430261D3E70000002701401902FEFF07
:106FA00010B586B0044614216846FEF714F90E4960
:106FB0002068884216D10D48416B42151143416348
:106FC000C16A01221143C162C06A6946104005903E
:106FD000022000900320019000200290052000076D
:106FE00000F068FA06B010BD002401400010024015
:106FF000F8B504464069254640350E4608280BD0B2
:107000002068C068C00709D0606D20210843606512
:10701000002028740120F8BD082700E00C2700F0AC
:1070200019FB009011E0701C0FD0002E05D000F06D
:1070300011FB0099401AB04207D9606D0421084342
:107040006065002028740320F8BD2068006838427D
:10705000E9D0606D01214902084360652068C1687C
:1070600009058A0F0C21002A1BD12022125D002A5B
:1070700017D10268120714D5826853070122002B2A
:1070800008DB43688B434360606D130298431043F1
:10709000606506E0606D202318436065A06D1043B5
:1070A000A065A069002801D1206801600020F8BD1A
:1070B00070B50446216800208968490721D4254617
:1070C0004035297C01291CD001212974E16901295D
:1070D00004D02046FEF762FD002811D1616D0A4AF6
:1070E0001140FF220132114361650021A16529741D
:1070F00022681C21116021688A6804231A438A606F
:1071000070BD022070BD0000FEF1FFFF30B50146EA
:1071100020314A790023022A04D00422C2630B7171
:10712000012030BD026814680E25AC43146002686B
:107130001468640864001460446C1C22144001222A
:107140001546006CA54045604A7118460B7130BD6C
:1071500070B50024014620314A79022A03D0042167
:10716000C163012418E0026813680E25AB43136065
:10717000026813685B085B001360436C1C221340B9
:10718000012215469D40036C5D604A7100220A7120
:10719000816B002900D08847204670BDF0B4016C97
:1071A0000D6801680C68466C1C2304221E401746BB
:1071B000B7402F420ED067070CD50C68A40602D446
:1071C0000C6894430C60416C19408A40016C4A6021
:1071D000016B1AE00227B74002462F402032002FF1
:1071E00017D0A70715D50C68A40605D40C680A2586
:1071F000AC430C6001215171446C02211C40036CB2
:10720000A140596000211171C16A002918D0F0BC59
:1072100008470827B7402F4212D0240710D50C6822
:107220000E25AC430C60446C01211C400B46A3406E
:10723000046C6360C163517100211171416BE4E71B
:10724000F0BC704770B504003CD01F48256814217D
:107250002818FDF74DFF800060641C48206402215F
:10726000204620300246417129681948E3680140F0
:10727000A06866691843236933431843A369184318
:10728000E3691843236A1843084328600121A06872
:107290008903884210D00D488030836A656C1C21B8
:1072A0000D400F26AE40B3438362656C63680D40AA
:1072B000816AAB400B4383620020E063012151717E
:1072C000107170BD012070BDF8FFFDBF00000240CD
:1072D0000F80FFFFF8B504468C4620300179002569
:1072E000012909D00126067141790027012905D01D
:1072F000077102252846F8BD0220F8BD0221417120
:10730000E76320680168490849000160614620463A
:10731000FFF796F8206B00282068016801D00E2244
:1073200005E0042291430160206801680A221143AC
:1073300001602068016831430160DBE770B50446F5
:1073400000F088F90546601C02D004480078241833
:1073500000F080F9401BA042FAD370BD500200201B
:10736000F8B51A4E0546307C0F46012807D001209B
:1073700030741748FFF7D8FA010002D021E002204C
:10738000F8BD0020C04338606C6814E02046FFF769
:1073900049FA0F48FFF7C8FA01460E484268082329
:1073A0009A434260426843159A434260002901D0E3
:1073B0003C6006E08034A8686A68C0018018A0427A
:1073C000E4D8002030740846F8BD0000B81300204F
:1073D00050C30000002002400548416802221143CA
:1073E0004160416801221143416000207047000064
:1073F00000200240F8B50C4C1646207C0F460128B0
:1074000008D0012020740948FFF78EFA00250028D3
:1074100002D006E00220F8BD65613E600348FFF738
:1074200083FA2574F8BD0000B813002050C3000093
:1074300011484168C9070BD0EFF3108172B60F4AAB
:10744000C2600F4AC26081F310884168C9070ED13B
:10745000416889070DD5EFF3108172B6094A0261C0
:10746000094A026181F310884068800701D5012034
:10747000704700207047000000200240EFCDAB892C
:1074800005040302BFAE9D8C1615141310B5C11F61
:10749000F93901D1FEF7D2FB10BD000010B5044947
:1074A0004A69024202D04861FFF7F0FF10BD0000B8
:1074B00000040140FCB500230124A2E027462A462F
:1074C0009F403A406FD04D68012D05D0022D03D06A
:1074D000112D01D0122D16D185680326AC465D0012
:1074E000AE46AE406546B543AC46CE687546AE4046
:1074F00065462E43866046680D79BE43ED06ED0F66
:107500009D4035434560C6685F000325BD40AE46DB
:10751000AE4335468E68BE402E43C6604E68022E8E
:1075200001D0122E14D1DE08B60036180196366A44
:107530005D07B446EE0E0F25B54000966646AE4395
:10754000B4460D69009EB54066462E43019D2E62ED
:1075500006687546AE430D79AD07AD0FBD403543A6
:1075600005604D68ED004BD5294D6E6B26436E636B
:107570009E08284DB6007519AC46AD689E07360FBB
:107580000F27B740BD4305273F07B84201D1002769
:1075900015E0214FB84201D1012710E01F4FB8423A
:1075A00002D102270BE02BE01D4FB84201D1032787
:1075B00005E01C4FB84201D1052700E00627B7407F
:1075C0002F436546AF60184D2E684F689643FF0302
:1075D00000D516432E606E684F689643BF0300D5F2
:1075E00016436E60AE684F689643FF0200D516439F
:1075F000AE60EE684F689643BF0200D51643EE605A
:107600005B1C0A681546DA4000D057E7FCBD000055
:10761000001002400000014000040050000800502B
:10762000000C0050001C005000040140006908409C
:1076300000D001207047426913460B401B04914360
:107640000B4383617047002A01D0816170478162DA
:107650007047000001488068704700005002002019
:1076600002488168027889188160704750020020C2
:1076700010B50848002401684022114301602046EB
:1076800000F00AF8002801D0012401E000F042FADD
:10769000204610BD0020024070B504460D4D7D20EF
:1076A0002978C000FDF724FD01460B480068FDF76E
:1076B0001FFD00F0C9FE002809D1042C07D20022CA
:1076C0002146401E00F03EFA00206C6070BD012093
:1076D00070BD0000500200205C020020704770471F
:1076E000F8B502F003FE714C0120A071607A401CD5
:1076F000C0B26072142808D9BFF34F8F6D496C482F
:10770000C860BFF34F8F00BFFDE76B4E7F25376822
:10771000ED05AF420ADAE08AFDF7BFFF01462846D1
:10772000FDF7CAFD3946FDF76EFD3060E08AFDF7D2
:10773000B4FF01467F20C005FDF7BEFD5F4D2968FF
:10774000FDF761FD286002F01FFF5D4801885D487C
:1077500003F022FE0120256BC005854201DA284690
:107760000BE0E08AFDF799FF01467F20C005FDF799
:10777000A3FD2946FDF79CFD2063FF21C9050025D7
:10778000C84200D32563A07800280BD102214E48BF
:10779000FFF74CFF02004D494D4817D00022FFF77C
:1077A00052FF656302214848FFF740FF494E002819
:1077B00055D065634848808AFDF76FFF3F4F3968B1
:1077C000FEF780F85ED2012030705CE00122D10328
:1077D0003F48FFF738FFE08AFDF75FFF01467F2053
:1077E000C005FDF769FD616BFDF70DFD3B49606369
:1077F0008842D7DD38480127F926403000900A2119
:107800003046FDF775FC002903D130493048FFF7B9
:10781000F3F802212C48FFF709FF002801D00027C8
:1078200001E0002F12D102212748FFF7FFFE0028B8
:107830000CD104F0F3FE00990120888004F09AFF37
:10784000642003F053FE1B491948C8600A2003F066
:107850004DFE3046761EF6B20028D0D1A2E7E08A6F
:10786000FDF71BFF01467F20C005FDF725FD616B7D
:10787000FDF7C9FC1A49606388429BDB0D490C483F
:10788000C86097E73570A089401EFDF7FBFE396898
:10789000FEF718F806D8E079002803D01149012036
:1078A0000870F8BD0F480570F8BD00000802002000
:1078B0000400FA0500ED00E04C0200204802002020
:1078C0004C0100205C0C00200004005000800000EF
:1078D00000000050760000203C04002000004040E2
:1078E0000000A0408600002070477047704710B528
:1078F000044600680168C943C90708D18168C943C3
:10790000C90704D1012141602046FFF7E9FE206844
:107910000168C943890708D48168C943890704D429
:10792000022141602046FFF7D9FE20680168C94363
:10793000490708D48168C943490704D40421416038
:10794000204600F0E5F820680168C943090708D41B
:107950008168C943090704D4082141602046FFF724
:10796000C3FF20680168C943C90608D48168C943B8
:10797000C90604D4102141602046FFF7B0FE2068FC
:107980000168C943890608D48168C943890604D4BB
:10799000202141602046FFF7A9FF20680168C94304
:1079A000490608D48168C943490604D4402141608E
:1079B0002046FFF79AFF10BDF8B5040005D0254614
:1079C0002035A87B002802D006E00120F8BD002069
:1079D0006873204600F03CF80220A8732068C26853
:1079E00084466368012B01D10620824316486169F1
:1079F000814202D0072040038243002B01D1D820CE
:107A000082431248A668024018463043676A266AD5
:107A10003E433043A66A30431043002B02D0012B73
:107A200004D005E02369E2691A4300E0E2681043EC
:107A3000054A914202D0A269114308436146C860D9
:107A40000120A8730020F8BDFFFF0000F8F119FF26
:107A500010B50068084988420CD10848816BC204FF
:107A600011438163002201210D2000F06BF80D20ED
:107A700000F05CF810BD0000007C004000100240E7
:107A80000068C06970470000F8B50446022025462A
:107A900020351746A8731D480268C3041A430260C4
:107AA0002068C2689B121A43C260206802690126DE
:107AB00032430261226810205060206881611021E9
:107AC000204601F0E3FB03281FD02168082048600E
:107AD000206847610821204601F0D8FB032814D014
:107AE000204601F063FBA87B03280ED02068816844
:107AF0003143816020680169314301612068016977
:107B0000042211430161AE730020F8BD000401405E
:107B1000704700000448416B012211434163816BAF
:107B2000020411438163704700100240002805DB06
:107B3000C106C90E01208840014908607047000055
:107B400000E100E010B503F019FA10BD0248016829
:107B5000821511430160704700700040F8B504467B
:107B600000780027534D800671D5524E403EB06BD1
:107B7000C00004D4B06BA9050843B06301274E4888
:107B80000168C90511D40168821511430160FFF72E
:107B900061FD009005E0FFF75DFD0099401A642843
:107BA00037D845480068C005F5D532680321090576
:107BB00060680A400140914208D08103890F03297F
:107BC00004D13168890301D50120F8BD2A69032158
:107BD00009040A4022D0084090421FD02078800635
:107BE0001CD528692A6988430121C9040A432A61EE
:107BF0002A698A432A612861C0050FD5FFF72AFD4B
:107C0000009008E0FFF726FD0099411A2B488142B9
:107C100001D90320F8BD28698005F3D56168880380
:107C2000800F032805D132680005824301400A43D2
:107C300032602869032261681204114008432861F8
:107C4000002F04D0B16B012000078143B16320787D
:107C5000C00705D0E868A168800880000843E86094
:107C60002078800705D5E8680C218843E16808433F
:107C7000E8602078400706D5E86803218902884338
:107C800021690843E8602078000706D5E8680321E9
:107C90000903884361690843E8602078000606D537
:107CA000E868032189048843A1690843E86000204B
:107CB000F8BD000040100240007000408813000032
:107CC000F8B50E46050038D05E480068C007C00F02
:107CD000B04214D25B4C2068400840003043206022
:107CE000FFF7B8FC074605E0FFF7B4FCC11B564898
:107CF00081427AD82068C007C00FB042F4D12878FA
:107D0000524C800705D5E068F0218843A9680843F4
:107D1000E0602878C00752D06868022806D003289F
:107D200007D0216801280AD0890504E02168890369
:107D300001E021688901002903DB0120F8BD490722
:107D4000F9E7E168890889000143E160FFF782FCF7
:107D50000746686802280AD0032814D001281ED0DC
:107D600029E0FFF777FCC11B374881423DD8E06826
:107D70000007800F0228F4D121E0FFF76BFCC11B44
:107D80003148814231D8E0680007800F0328F4D1E0
:107D900015E0FFF75FFCC11B2B48814225D8E06846
:107DA0000007800F0128F4D109E0FFF753FCC11B45
:107DB0002548814219D8E0680007800FF5D1214895
:107DC0000168C907C90FB14217D9016849084900BC
:107DD00031430160FFF73EFC074608E005E0FFF78E
:107DE00039FCC11B1848814201D90320F8BD154850
:107DF0000068C007C00FB042F1D12878400706D50F
:107E0000E068072109028843E9680843E0602878B0
:107E1000000707D5E0680721C90288432969C9001E
:107E20000843E06000F03AF8E168094A0906090FE2
:107E3000515CC8400749086007480068FFF72CFC00
:107E4000F8BD00000020024088130000001002402E
:107E500084CA00085C02002054020020044805493E
:107E60000068C968044A4905490F515CC840704719
:107E70005C020020001002409DCA00080448054929
:107E80000068C968044A8904490F515CC8407047BA
:107E90005C020020001002409DCA000870B51A4A1A
:107EA000D3681A490C2018408D0004280CD04E00CD
:107EB000082810D00C2810D050680004410F012071
:107EC000C003491C884070BD1068C00601D5084633
:107ED00070BD284670BD304670BD98020C4C000F36
:107EE000205C1B029C0FD368641CDB0301D5314668
:107EF00003E01268D20600D4294603F01AF822469D
:107F00000023FDF71FF970BD0010024000093D007D
:107F100094CA0008FEB505007ED0FE4CE7680C2030
:107F2000E66807400120000406402878C00747D0D3
:107F3000082F05D00C2F0AD101200004864206D15B
:107F4000206880033CD568680028E5D038E001202F
:107F500069680004814203D121680143216011E076
:107F6000052301221B0492049942216802D1114386
:107F70002160F1E781432160216801400091206880
:107F800090432060686800280DD0FFF763FB0090E5
:107F900005E0FFF75FFB0099401A64287BD8206852
:107FA0008003F6D50CE0FFF755FB009005E0FFF7E6
:107FB00051FB0099401A6428F0D820688003F6D459
:107FC0002878800756D50923E868042F0DD00C2F98
:107FD00001D1002E09D000283CD0216899430143EB
:107FE0002160FFF737FB064628E02168490701D5E5
:107FF000002891D061681F22120291432A6912025F
:10800000114361602168994301432160FFF746FFF6
:10801000E16809060A0F00E08BE1BF49895CC840AE
:10802000BE490860BE480068FFF736FB002873D1E0
:1080300020E0FFF70FFB801B0228AFD82068400725
:10804000F7D560681F21090288432969090208439E
:1080500060600FE02068400840002060FFF7FAFAF7
:10806000064604E0FFF7F6FA801B022896D820683F
:108070004007F7D42878C00660D5002F0CD0A86937
:1080800000284AD02068FF21013108432060FFF713
:10809000E1FA06462EE0C1E02068800502D5A86915
:1080A0000028A6D06068072149038843296A08434D
:1080B00060606068297F0002000A0906084360606A
:1080C000286A410B0120C003491C8840E168090669
:1080D0000A0F9149895CC84090490860904800683F
:1080E000FFF7DAFA002817D128E0FFF7B3FA801B70
:1080F0000228A2D820688005F7D5606807214903C7
:108100008843296A084360606068297F0002000A8A
:1081100009060843606011E0E2E02168FF200130B9
:1081200081432160FFF796FA064604E0FFF792FAD2
:10813000801B022872D820688005F7D42878794EF1
:10814000000724D568690028306910D00121084350
:108150003061FFF77FFA009005E0FFF77BFA0099A6
:10816000401A02285AD830698007F6D50FE0400837
:1081700040003061FFF76EFA009005E0FFF76AFA01
:108180000099401A022849D830698007F6D4287827
:10819000400766D500200290A06BC00006D4A06BFB
:1081A000012109070843A063012002905E4801688D
:1081B000C90511D40168821511430160FFF74AFA1D
:1081C000009005E0FFF746FA0099401A642825D888
:1081D00055480068C005F5D5FF20AA6801308242E5
:1081E00003D131690143316111E001218902002A83
:1081F00007D005231B029A4203D132690A43326138
:10820000EFE7326982433261306988433061A868A0
:10821000002810D0FFF71EFA009008E05FE0FFF79B
:1082200019FA01460098091A4048814257D8306926
:108230008005F4D50DE0FFF70DFA009006E0FFF79A
:1082400009FA0099411A3948814248D830698005B5
:10825000F5D40298002804D0A06B012109078843B7
:10826000A063686A002866D00C2F3ED0012636062F
:108270000228206805D0B0432060FFF7EBF90546DF
:108280002FE0B0432060FFF7E5F9074604E0FFF771
:10829000E1F9C01B022822D820688001F7D4E96ADE
:1082A000A86AE2680843296BFD231B049A43114323
:1082B0000843E060206830432060FFF7CBF90546B3
:1082C00004E0FFF7C7F9401B022808D820688001A6
:1082D000F7D530E0FFF7BEF9401B022801D9032093
:1082E000FEBD20688001F5D425E00128F8D0E068C3
:1082F00001210904AA6A014091421AD10F2189047F
:10830000EA6A0140914214D1032189050840296B92
:1083100088420DE00010024084CA00085C02002080
:1083200054020020401002400070004088130000FA
:1083300001D00120FEBD0020FEBDF8B504000ED026
:10834000FF27606A0537002500280AD0256165618E
:1083500026464036A562707C002807D00AE001203E
:10836000F8BD6068B842F3D0E561F1E735742046A6
:1083700000F03EF8022171742068026840239A439D
:1083800002602123A26860689B021A4038401043B3
:10839000E3688A021340184323690B40217D184388
:1083A000C907C90F0843A169931019400843E1693F
:1083B000382319400843216A802319400843A16AE1
:1083C00093001940084321680860A0690421000C4B
:1083D0000840616A102319400843216848602068FA
:1083E000C1699143C1616565012070740020F8BDC9
:1083F00010B586B0044614216846FCF7ECFE10491F
:108400002068884219D10F48416B8214114341639F
:10841000C16A01221143C162C06A00211040059067
:10842000E02000900220019003200390029104912B
:10843000052069460007FFF73DF806B010BD0000B3
:108440000030014000100240094910B5401E88422A
:1084500001D9012010BD074C60610321081F02F003
:108460008DFD0020A06107202061002010BD0000CC
:10847000FFFFFF0000E000E0F0B502462032137E6F
:10848000012B1ED0012515760223537606687468E9
:10849000B3687027BC430F68274377600068AC0758
:1084A000A04205D0084CA04202D0084CA04204D102
:1084B00080244968A34319438160557600201076D3
:1084C000F0BD0220F0BD0000000801400014014092
:1084D00070B5050005D02C462034607E002802D0FF
:1084E00006E0012070BD00202076284600F010F83C
:1084F00002206076291D286801F06EFF0120A07718
:10850000A076E076207760776076002070BD00006E
:10851000006801218907884204D10348816B012248
:10852000114381637047000000100240F8B5054612
:1085300004462035287E012817D001262E760220F9
:108540006876226890687727FF23B8431B02984318
:1085500090600A68502A31D00EDC202A4BD006DC0D
:10856000002A48D0102A3AD145E00220F8BD302A2E
:1085700041D0402A33D136E0602A27D0702A12D069
:1085800001200003121A2AD0824228D1CB684A68FF
:108590008968206801F059FF2068816801229203F0
:1085A000114381601BE0CB684A688968206801F04C
:1085B0004CFF216888683843886010E0CA684968C1
:1085C000206801F0BCFF5021206806E0CA684968B5
:1085D000206801F0C5FF6021206801F041FF6E7640
:1085E00000202876F8BDCA684968206801F0A7FF16
:1085F00040212068F1E711462068EEE710B586B00B
:10860000044614216846FCF7E6FD0121206889072D
:10861000884212D10A49CA6A02200243CA62C96A60
:1086200001900140059141020091002102910391C6
:10863000049069460348FEF73DFF06B010BD0000F8
:108640000010024000040050F8B5064604462036EB
:10865000307E0D4601280BD0012008273076002AF5
:1086600008D0042A16D0082A2AD00C2A4DD137E087
:108670000220F8BD206801F0FBFE206881693943C3
:108680008161206881690422914381612068816948
:10869000EA6812E0206801F003FF20688169012286
:1086A000D2021143816120688269012189028A43D3
:1086B000826120688169EA6812021143816124E0C5
:1086C000206801F006FF2068C1693943C161206854
:1086D000C16904229143C1612068C169EA6812E05E
:1086E000206801F011FF2068C1690122D202114304
:1086F000C1612068C269012189028A43C261206880
:10870000C169EA6812021143C16100203076F8BDE8
:1087100070B5050005D02C462034607E002802D0BC
:1087200006E0012070BD00202076284600F00FF8FA
:1087300002206076291D286801F04EFE0120A077F6
:10874000A076E076207760776076002070BD704775
:1087500070B505462C4602202034002908D0042993
:108760000BD008290ED0627F012A10D0012070BDE5
:10877000A27E012AFAD1A0760AE0E27E012AF5D192
:10878000E07605E0227F012AF0D1207700E06077D3
:108790000122286801F04CFE01222868920701217D
:1087A000904205D0074A904202D0074A904204D135
:1087B00082685207520F062A02D002680A430260FA
:1087C000002070BD000801400014014070B504464F
:1087D0000D460068002201F02BFE2068016A0C4A59
:1087E000114203D101684908490001600120203489
:1087F000002D06D0042D06D0082D06D0607700206D
:1088000070BDA076FBE7E076F9E72077F7E7000098
:10881000111100007047704770470000F8B50268FA
:108820000446D06911689668814B05461D40202397
:10883000002D6CD0F7077F4DFF0FBC460D402F4336
:1088400079D02546C7078035002F06D0CF0504D53F
:10885000012717622A683A432A60820708D5F2077F
:1088600006D0276802223A622A6804273A432A601F
:10887000420708D5F20706D02668042232622A6829
:10888000022632432A6002070AD50A461A40664683
:10889000324305D02668082232622E6816432E60C5
:1088A000020508D54A0106D501222668D2023262A5
:1088B0002A681A432A602A68002A30D0800606D522
:1088C000880604D5616E002901D0204688472868B3
:1088D00021688968490602D42821084225D020460B
:1088E00002F053F820688168490619D58268402152
:1088F0008A438260206F002812D04F498163206F25
:10890000FEF726FC00280AD0206F816B06E0850662
:1089100011D58D060FD5616E77E020468847F8BDEA
:108920002046FFF779FFF8BD05E02046FFF774FF0A
:1089300000202860F7E7256E012D56D1C50654D5D5
:10894000CD0652D510261662206881682546490654
:10895000403500292ADA226F116849680904090C98
:10896000E1D02F8B8F42DED96983116809688906AF
:1089700017D4016832019143016020688168490879
:108980004900816020688168402291438160E367EB
:108990000020206620680168B1430160206FFEF767
:1089A000B5FB288B698B401A81B21AE0298B6A8B40
:1089B000891A6A8B89B2002AB5D00029B3D002681F
:1089C000FF252135AA4302602068826852085200C0
:1089D0008260E36700202066606620680268B24318
:1089E00002602046FFF716FF9DE7C50208D5750215
:1089F00006D50120000510622046FFF70CFF92E724
:108A0000050605D50D0603D5A16E002985D18AE797
:108A1000400688D5480686D5116820464024A143E3
:108A2000116083670021816600F043F97BE7000055
:108A30000F08000020010004B1A8000810B50400D0
:108A400003D0A06F002802D007E0012010BD002154
:108A500074200155204600F027F82420A0672068E4
:108A60000168490849000160204601F0E1FF012842
:108A7000ECD0606A002802D0204601F003FE206896
:108A800041680922D20291434160206881682A220C
:108A900091438160206801680122114301602046F2
:108AA00001F056FE10BD0000F0B587B00646142157
:108AB0006846FCF790FB2C493068884251D12B481E
:108AC000416B0122920311434163C16A01221143A8
:108AD000C162C06A0025104005900320400200904A
:108AE0000220032701A9A1C10420049005206946A2
:108AF0000007FEF7DFFC1F4C1D48A560E56081C440
:108B00008027E560A7602020256160610002A061E8
:108B10001848083CFEF796FB002801D0FDF780FEC0
:108B20003467A662144C1248214614382060032092
:108B3000606010200831A1C16561A561E561204632
:108B40002562FEF77FFB002801D0FDF769FEF46681
:108B5000002201211B20A662FEF7F4FF1B20FEF776
:108B6000E5FF07B0F0BD00000038014000100240F2
:108B700030000240281300207013002070B5C36F2E
:108B8000202B27D100290BD0002A09D0012483688B
:108B90002403A34206D10369002B03D1CB0701D0E4
:108BA000012070BD034660331C7D012C12D00124CE
:108BB0001C7500230366084C0368A34207D05C6859
:108BC000240204D51C680125AD062C431C6002F06C
:108BD0002FF870BD022070BD0048004070477047FC
:108BE000FFB50446806F83B017460D4620285ED13E
:108BF000002D0AD0002F08D0A168C001814207D102
:108C00002069002804D1E80702D0012007B0F0BD98
:108C1000204660300090007D012848D00098012156
:108C200001750020802108512120A067FEF712FD68
:108C3000264640360190378277820120A1680003E2
:108C4000814202D12069002805D02F4600250099D5
:108C50000020087511E00027F9E700228021204656
:108C600002F02CF8002815D1002F15D02168387893
:108C700088627F1C708A401E7082708A019B002867
:108C800006980090E9D100224021204602F016F813
:108C9000002808D00320B9E728882168C005C00D46
:108CA0008862AD1CE6E72020A0670020AEE7022026
:108CB000ACE77047034D044C04A002F013F9E560E3
:108CC000FAE700000400FA0500ED00E04861726474
:108CD0004661756C745F48616E646C65722E0D0A36
:108CE0000000000010B505242407002204212046BE
:108CF000FEF7A9FC002208212046FEF7A4FC0A206A
:108D000002F0FBFB012204212046FEF79CFC0A2016
:108D100002F0F3FB002204212046FEF794FC10BD74
:108D200010B505242407002204212046FEF78BFC01
:108D3000012208212046FEF786FC0A2002F0DDFB16
:108D4000012204212046FEF77EFC0A2002F0D5FB1A
:108D5000002204212046FEF776FC10BDF8B5002461
:108D60000526074625463607002204213046FEF731
:108D70006AFC0A2002F0C1FB012204213046FEF702
:108D800062FC6006040E08213046FEF74FFC002806
:108D900001D0641CE4B2052002F0AFFB6D1CEDB203
:108DA000082DE1D3002F03D0FFF79CFF2046F8BD2C
:108DB000FFF7B6FFFAE770B505260546360700222D
:108DC00004213046FEF73FFC0024E80901D00122CF
:108DD00000E0002208213046FEF735FC6806050E4B
:108DE0000A2002F08AFB012204213046FEF72BFC08
:108DF0000A2002F082FB002204213046FEF723FC09
:108E00000A2002F07AFB641CE4B2082CDDD370BDAA
:108E100010B505242407012208212046FEF713FC83
:108E2000012204212046FEF70EFC002208212046E4
:108E3000FEF709FC0A2002F060FB00220421204614
:108E4000FEF701FC10BD10B5052424070022042103
:108E50002046FEF7F8FB002208212046FEF7F3FB30
:108E60000A2002F04AFB012204212046FEF7EBFB18
:108E7000012208212046FEF7E6FB0A2002F03DFB16
:108E800010BD70B505252D070024012208212846B4
:108E9000FEF7D9FB062002F030FB01220421284610
:108EA000FEF7D1FB062002F028FB07E0641CE4B2C9
:108EB000FA2C03D9FFF7C7FF012070BD082128460F
:108EC000FEF7B4FB0028F1D1002204212846FEF76A
:108ED000BAFB002070BD0000F8B501F06BFC01F09A
:108EE0009BFC3D480068C069FDF78AFD3B4D6883E7
:108EF000FDF758FE3A4E28700121C9023046FEF7B0
:108F000095FB77010024002827D036480460A87A12
:108F1000002803D10120A87201F04CFF80213046C7
:108F2000FEF784FB002806D0002208213046FEF719
:108F30008AFB012205E0012208213046FEF783FB6F
:108F40000022052039460007FEF77DFB264D274EFF
:108F5000A88C274F012803D01CE0AC720022EBE75D
:108F600024486946088072B680212348FDF770FCCA
:108F7000002804D0022269461F48FDF70DFD62B6A5
:108F80001EA001F0AFFFAC8403F0F4FB642002F0FC
:108F9000ADFAFE60688C012809D113486C84403812
:108FA000048003F0E7FB642002F0A0FAFE60288C46
:108FB000012806D12C8403F0DDFB642002F096FA30
:108FC000FE600948114A40380188914202D1C088A8
:108FD000002800D1FE60F8BDDC110020080200204E
:108FE00000040050480200207C0400200400FA0520
:108FF00000ED00E0AAAA0000384A0008BDF8C8EB5E
:10900000C9FDBCB6C4A3CABD0D0A0000AA55000024
:1090100010B53721202000F070F80321212000F046
:109020006CF84021222000F068F80821232000F08D
:1090300064F8AA21302000F060F80A480221018774
:10904000322000F05AF80121332000F056F85F2159
:10905000202000F052F8044800F008F80A2002F03E
:109060004CFA10BD3C0400200300002010B501465E
:109070000F2000F021F8002800D0012010BD10B50D
:109080000446FFF7C5FE3220FFF795FEFFF7F9FE15
:10909000E0B2FFF790FEFFF7F4FEFFF7B9FE3320D2
:1090A000FFF789FEFFF7EDFE0020FFF757FE0446AD
:1090B000FFF7C9FE204610BD10B50C46FFF7DFFFD5
:1090C0002070012010BD70B50D460446FFF7A0FECC
:1090D0003220FFF770FEFFF7D4FEE0B2FFF76BFE21
:1090E000FFF7CFFE2846FFF766FEFFF7CAFEFFF741
:1090F000AAFE0A2002F001FA70BD10B5FFF7E3FFE7
:10910000012010BDF8B5214F43883B83C4887C8380
:109110000289BA838189F983408938845B43644337
:109120001819524380184943FBF7F8FFFCF7BCFAC3
:1091300003F08CF80022164BFCF7AEF9154A164BDB
:10914000FCF79CF93E46803671633063F88B4043F0
:10915000FCF7AAFA04460D46388CFCF7B9FA11223E
:10916000FCF77AFA22462B46FCF7FEF903F06EF87C
:109170000022074BFCF790F9064A074BFCF77EF9F3
:10918000F163B063716C306CF8BD000040010020E9
:10919000000024408FC2F5285C6F5E4010B5024885
:1091A000FEF7A5FB10BD000014110020FEB504461B
:1091B000002772B6334A01688B1804D13248C76859
:1091C00003208004074088680190C86800904869BF
:1091D0008E69002B08D12C4940398B6ACD042B4372
:1091E0008B628B6AAB438B62014631433CD025498D
:1091F0002368CB4205D12449CA6803239B049A43C0
:10920000CA6025462035002810D021680A6901234C
:109210001A430A61216848610821204600F036F8A7
:10922000032800D1A873216808204860002E10D0C0
:1092300020680169012211430161206886611021C3
:10924000204600F023F8032800D1A87321681020DD
:1092500048600C482168C14206D10B48C16803220E
:10926000920491433943C16020680169490849006B
:10927000016121680198886021680098C86062B621
:10928000FEBD00000084FFBF4010024070B50646DE
:109290000B480D46002409490068FBF729FF7D2192
:1092A000C90048433168401E00D103240B682A4698
:1092B0009A4301D00028F6D1204670BD204E000010
:1092C0005C0200201CB5002116480091144A01914F
:1092D0000260C1631205426081600722826301223D
:1092E00002610246C16020321170FF235170C23307
:1092F00043628162117301638161042241634261AF
:10930000C161FDF769FD084800908013019069462E
:109310000448FDF711FD00210248FDF7B7FC1CBD14
:1093200000240140B81000200200000408B50848DD
:10933000016B012211430163006B01211040009079
:1093400000220A20FEF7FEFB0A20FEF7EFFB08BD15
:1093500000100240F0B587B014216846FBF73BFFD0
:109360005048C26A04210A43C262C26A0A40059296
:10937000C16A80273943C162C16A39400591C16A17
:1093800001252943C162C16A29400591C16A0226AB
:109390003143C162C06A2A463040059005201C2135
:1093A0000007FEF750F901223F494048FEF74BF90C
:1093B00000223F493D48FEF746F991210520002251
:1093C00009020007FEF73FF93A4801900024052002
:1093D0006946009502940007FEF76CF80C20009097
:1093E0001120019003200390052002946946000794
:1093F000FEF760F81020009005206946039601955D
:1094000002940007FEF756F8112001900294694675
:10941000009503942548FEF74DF8274801906946CA
:10942000009602952148FEF745F8E8026A4651C2C7
:1094300069461E48FEF73EF82048009002946946AF
:10944000019503941948FEF735F891200002009029
:10945000052002946946019503940007FEF72AF857
:1094600069461248009702950194FEF723F82802F6
:10947000009010480190694602940C48FEF71AF8D3
:10948000002201210520FEF75DFB0520FEF74EFBC3
:10949000002201210720FEF755FB0720FEF746FBBF
:1094A00007B0F0BD001002400102000000040050AF
:1094B00008300000000011100000211008320000E8
:1094C00010B50F4C0D482060FF2005306060002073
:1094D000A060E06020616061E061012120624902DA
:1094E0006062A161A0620720E0622046FEF725FFCE
:1094F0002068016840221143016010BD0030014026
:109500004411002010B58AB00024049405940694F8
:109510000794089401211848099400940194029436
:109520008907039401600921846041600461134943
:109530004461C160FEF7CCFF01200003049004A940
:109540000D48FEF7F3FF0C48FFF7E2F8089408A96E
:1095500009480994FEF790FF6020009008480190A8
:1095600002940822694603940348FFF76DF8024805
:10957000FFF744F80AB010BD9C11002093040000CE
:109580005702000000B585B014216846FBF723FEA2
:109590000E480D490160E1214902416000218160CE
:1095A000C160016181610C22C161426101623021AF
:1095B00041620121090381634900C163FFF73EFA5B
:1095C00001F0F2FB05B000BD00380140DC110020C5
:1095D00070470000F0B589B00A2002F00DFB7D2035
:1095E000400102F023FBFF4C0025A570FE48606699
:1095F000607C0C2801D30B20607461790A200A2951
:1096000000D96071E570217D002904D0032902D0C2
:109610000121617600E06576F449F54E09783171F3
:10962000F44AA179127849001143A27DF24F9200C9
:109630001143627E52011143F171216CF1700A0AEB
:109640003272491C216439880A2900D9388061792D
:1096500038884A000818A087B074E548E7491330F5
:10966000FBF7A0FD3888E649420060794000801988
:109670001330FBF797FD607939888200401840006D
:10968000DE49801962311330121DFBF78BFD6079C2
:109690003988421852008000101880198A00D94970
:1096A0001730FBF77FFDA08F0C2142004843801943
:1096B000D5491730921CFBF775FD3020205E00283D
:1096C00003D0D249098A0818208616207072D04823
:1096D000C4490078B072E08C3073C548203113382B
:1096E0000A7A0275497A4175A08F0022C0001D30A8
:1096F00080B2BF4902F06AFBA08F0021C0001D307C
:1097000080B202F075FBC348FEF7BAF90127608505
:10971000BF0309E0BF48FEF7B3F980B26085218F2F
:10972000FF392D39884206DB218F80B28842F1D380
:10973000C9198842EED8022002F0AEFAAC480126E0
:10974000C571A574A5732674E573B248FEF798F940
:10975000A0850746E570A08FFBF7BAFFAE4AAF4B76
:10976000FBF79AFE01F05EFE0022AD4BFBF7E2FD37
:10977000FCF70AF80006C10CC81980B2F103E085B5
:10978000884201D3401AE085A64820652079401C14
:109790002071A048FEF774F9984F6085963F3846CF
:1097A00022300690001F0290001F0190801E03903F
:1097B00072E19848FEF764F960850BE09548FEF782
:1097C0005FF980B26085E18D884203D3964A89189B
:1097D000884207D300210F2002F044F993496064C6
:1097E0000842EBD0606C411C20D040047ED5812221
:1097F000D20100210F2002F0BEFA0021102002F059
:1098000031F941067D48490E00229638216602F062
:1098100097F902F03BF9A067002002F007FA002058
:1098200002F0A7F9797A1729C2D101E001F0C8FB4B
:1098300002227F49781DFBF7D9FC0028B8D102F03D
:1098400047FB684A803203C202F01CFB654A803243
:10985000D1609060E0786949401CE0709D390A7AD7
:1098600068460270497A417000880790218D8842CD
:109870007ED16249032092310870069800905948C1
:10988000029A803083680020019900F0A1FC5849B9
:1098900068488C31C98E0180554952488C31098FF6
:1098A00081845C48FEF7ECF8608501F089FFF87C64
:1098B0000009607513D002225D49781DFBF796FC04
:1098C00000280CD14A48A674C671206E4B49163840
:1098D000C2B24A48E27480399E30FBF763FC022131
:1098E0005548FDF7A3FE002814D000E0C7E0002093
:1098F00040490870414862300068E0642065606556
:10990000F97C0907090F032900D02175216E26294A
:1099100002D019E00120EBE73549324A8C31C98F7A
:109920005186394A039B143A1B88938288420ADD88
:10993000002808DD002906D0E17D481CE0750529D6
:1099400002D9257000E0E5752571A673E673A08C39
:109950003A49FF30C33080B2A08488420ED94942D0
:109960004018A08433480188491C89B2018000E076
:109970000FE07D22D200914200D305802D487D2149
:109980000088C9004843A18C4018A06500F04AFC3B
:109990008BE0FDF71DF80590069800901149059899
:1099A0008031401C8B68C0B2029A019900F010FC13
:1099B00012490598923103220818427005983039EF
:1099C0008000009040184068E064206E262806D190
:1099D00005980D49400041180398008848800749C0
:1099E00032312DE0700000203F420F0008020020BD
:1099F00078050020440200204C010020C20600200F
:109A0000C40B00205C0C0020780800207C0400209F
:109A10001E020020141100209A9999999999E13F0A
:109A200000000840A0860100983A000000D02724DA
:109A3000340200204002002000040050E703000030
:109A400000984018F039898F0180684900984018C3
:109A500067491630CB688A6802F0FDF9E16C606EE8
:109A6000814219DA6348009A8058002814D00128EE
:109A700001D0884210DD6166079804900CE05E4AD0
:109A800000210F2002F077F96079E178401C8142D3
:109A900002D0002002F06DF8618DE08D814200D28D
:109AA00087E6564A80188142FAD8A07B012801D067
:109AB0000220A07301F084FE4F4A00210F2002F023
:109AC0005AF9217900291CD020460A2906D90571A6
:109AD0002670FCF7CBFC2079002802D0002000F093
:109AE0000BF9FCF7D9FBA07C00285CD041496C3114
:109AF0000B78A372487860728A782272022B17D092
:109B000051E0206D616E323881420FDAE1792046F2
:109B1000491CC9B2E1710229E3D9C57104990185D3
:109B2000022101706573FCF787FFD4E7E571D8E780
:109B300010280ED0324B062815D0C82833D218185A
:109B4000C91CFBF72FFB02F015FE642001F0CEFCD0
:109B50006CE62C4F38684000000E24D1C878FBF723
:109B60009CFD38601FE026480F460222C91C801D5C
:109B7000FBF73CFB002816D02148627AF91C8018BC
:109B8000227AFBF70FFB02F0F5FD1D48C1887D200E
:109B9000C000FBF7ADFA1C4908800146C820FBF75E
:109BA000A7FA1A4908800027022613E01148114934
:109BB0007D0032381A39405B495B884208D02670F4
:109BC000FCF73AFF002060730A4901204A394853E4
:109BD0007F1CFFB260798742E8D3074A00218032B8
:109BE0000F2002F0C8F809B0F0BD00007805002091
:109BF000F0000020F406002000D02724983A00004E
:109C00003C040020380200201E0200202C0200200C
:109C1000F8B52E4C0546206F2D4A281A411E606764
:109C2000914215D21A21615E081AFBF73DFD294ABF
:109C3000294BFBF731FC064634200F46205EFBF72C
:109C400033FD32463B46FBF775FBFBF779FDA086FB
:109C5000002020761D481C23C35EC28C1F4800884C
:109C600084461F4806881DE06046484380181D4F03
:109C700080B23880302778436427643078431A4FA5
:109C8000A066C01985420BD2C8B218493422088098
:109C9000A06EA25E411BC9188918E1662067F8BD55
:109CA000491C2176217EB142DED330204243104848
:109CB0006421101848430F4941182167A0663421D8
:109CC000401B615EC0184018E066F8BD70000020BF
:109CD000CF0700009A9999999999B93F2C020020D1
:109CE0001E0200204202002078ECFFFF2A02002022
:109CF00074270000C0BDF0FFFEB5294D2988491C1E
:109D00008FB228492F800E88FBF7CEFC264A274BBE
:109D1000FBF7C2FB0191009025483146FBF7E8F9BB
:109D2000244C618F4218B74206D300202880224875
:109D3000019E1018009D02E01046019E009DFBF759
:109D4000C7FC33462A46FBF7F5FAFBF71DFDE08614
:109D5000012580B2ED03A84201D3401BE086E08BD1
:109D6000FBF7B6FC154A164BFBF7FEFB0646E08EEA
:109D70000F460090FBF7ACFC32463B46FBF7DAFAA5
:109D8000FBF702FD80B22087A84201D3401B208749
:109D90000C4900980968486100986087FEBD000082
:109DA0002A0200201E0200201904560E2D62404097
:109DB000E17A0000700000201F050000F853E3A5C1
:109DC0009B843E40141100207047000070B532495A
:109DD0003048086002F022FC304800F0B9F9304CFD
:109DE000A0832E48801C00F0B3F9E0832B48001DAF
:109DF00000F0AEF920842C4D2A4868802846403077
:109E00000179A170294AE98E1170E98FE171A98F5A
:109E1000217280796070A87A6071AE880521E6624F
:109E20002182E888FBF764F9608201463046FBF73F
:109E30005FF98800081886B27D213046C900E681A6
:109E40004843FBF745FC1A4A1A4BFBF78DFBFBF71F
:109E50009BFCA0822683E18AC820FBF749F9A084F5
:109E600001206084FCF7CCFD6083688FA081E988C5
:109E70007D20E184C000FBF73BF9E082A28A0E4915
:109E80000E48FDF701FE6888C2B2010A0CA001F07D
:109E900029F870BDD5AD000868000020004F00080B
:109EA000080200200B0200003C04002018000020E3
:109EB000F853E3A59B843E40FF7F0000141100206F
:109EC000B9CCBCFEB0E6B1BE3A5353CBABC2B7B6C9
:109ED000A8CEBBB1EAC7A92DB7C0D7B2BBF9D5BED2
:109EE000205625642E25642E200D0A00F8B5744CEA
:109EF0000026744D2671012028807349C8200880EF
:109F0000E07A401CE072C00706D0E08C411EE1847C
:109F1000022801D2C820E0840120C043FFF7ECFEF4
:109F20000A2001F069FE7D20400101F07FFE022140
:109F30006648FDF77BFB00283CD000206449800088
:109F40000978654F49000843624909780843B872A7
:109F5000102078726148C1887D20C000FBF7C8F8E6
:109F600078735F485D490078B87338460B308A785B
:109F70000270C9784170411C58482030027ECA7076
:109F8000407E087155482230027E4A71407E8871B9
:109F9000544855490078C87400223946172001F00A
:109FA00015FF0021172001F023FF022001F074FEAD
:109FB0004E4F03E00120C1E7FEF78EFF00210F2086
:109FC00001F050FD38426064F6D0606C411C74D0E2
:109FD000400470D58122D20100210F2001F0CBFE78
:109FE0000021102001F03EFD41063B48490E0022B1
:109FF000B430216601F0A4FD374FB437787A1128C8
:10A0000059D102223A49781DFBF7F0F8002852D1C5
:10A01000F81F027A69460A70407A4870B97A298036
:10A02000C820FBF765F82849324D0880387BE0846A
:10A0300038462838C08E2880394621482839098F6B
:10A0400081842D48FDF71CFD6085A08C2B49FF30D5
:10A05000C33080B2A08488420BD949424018A08402
:10A0600028882649401C80B20B312880884200D3C2
:10A070002E8028887D21C9004843A18C4018A06506
:10A0800000F0D0F86846008820851349B87CC731B5
:10A090006071420008460D468330FBF783F8607913
:10A0A000294642001048D638FBF77CF8E08CFF28A0
:10A0B00001D001202070F8BDFFE700F081FF000013
:10A0C000700000201E0200202C020020000400501E
:10A0D0000F02002010020020780500203C04002020
:10A0E0001800002008020020B007002000D027241C
:10A0F000340200204002002014110020E703000079
:10A1000070B586B014216846FBF765F801250F4E3F
:10A11000ED03002229463046FDF795FA0120002480
:10A12000019002946946009503943046FDF7C2F908
:10A130000320019002946946009503943046FDF790
:10A14000B9F9022001F0D2F906B070BD0004005048
:10A150000088704770470000F8B5044600206A4642
:10A160001080194D55222A70AA226A700322AA7003
:10A17000661DEE702A716971144A49008918AC7124
:10A180002246E81DFBF70EF8002007E029186A4672
:10A190008978128889186A461180401CB042F5DB24
:10A1A000611DA81CFCF716F90146684601802919B3
:10A1B0000078C87168464078087221460931024823
:10A1C00000F004FCF8BD0000BA0900203C040020A7
:10A1D000FFB505468400114881B01E4620180422B0
:10A1E0000A9FFAF7DFFF0D4804222C30201803994C
:10A1F000FAF7D8FF09480949583020180660680066
:10A20000B0314018397801707978417004480349B9
:10A21000806F8431085105B0F0BD00009008002027
:10A2200070000020FEB5FFF7F3FC2548FDF728FC81
:10A23000244C86B2668560790A21081AC000FBF7B3
:10A2400033FA07460191E06EFBF742FA1E4A1F4BB4
:10A25000FBF78AF900900D463046FBF739FA2B469A
:10A26000009AFBF767F83A46019BFBF763F8FBF7A8
:10A270008BFA85B2E586E08BFBF72AFA124A134B7C
:10A28000FBF772F906460F462846FBF721FA3246DD
:10A290003B46FBF74FF8FBF777FA81B20120C0038A
:10A2A0002187814201D3091A2187854201D3281AC7
:10A2B000E0860349E08E096848616087FEBD0000C2
:10A2C0001411002070000020F853E3A59B843E4049
:10A2D000034A1168382389B29943014311607047DA
:10A2E0000030014010B5FDF7BBF910BD10B59AB0B4
:10A2F00034216846FAF76FFF14210DA8FAF76BFFB7
:10A300001C2112A8FAF767FF1B4801680324E40226
:10A31000A143C21489180160FDF718FC17480169B0
:10A32000A143016106200090FF200130029001202E
:10A330000390102004900220099040040B9000012B
:10A3400000240C900A946846FDF7E4FD0F200D9060
:10A3500003200E900F941094012111940DA8FDF785
:10A36000AFFC81201290032080041890149412A84E
:10A37000FDF7F4FB1AB010BD007000404010024021
:10A3800010480168821511430160C1680E4A1140EE
:10A39000C16001680D4A11400160816849084900A7
:10A3A000816001680122920491430160C168FD222D
:10A3B00012049143C160002101610649044888608C
:10A3C00070470000001002400C40FF88F6FFF6FEC8
:10A3D0000050000800ED00E070B5026801239B0703
:10A3E000114C124D984203D0A04201D0A84203D193
:10A3F0007026B2434E683243984203D0A04201D047
:10A40000A84204D103231B029A43CB681A4380233A
:10A410009A430B691A4302608A68C26209688162C2
:10A420000121416170BD000000080140001401409D
:10A4300010B5CB06DB0E0121046A99408C430462FF
:10A44000016A9A401143016210BD30B58468FF254E
:10A450002D021B021343AC430B432343836030BDE7
:10A46000826870239A430A4307210A438260704737
:10A4700030B5026A520852000262026A4568836976
:10A480007024A3439C080B68A40023430224A24326
:10A490008C6845601443836149684163046230BD40
:10A4A00030B5026A10239A430262036A45688269E2
:10A4B00073242402A2430C682402144320229343F1
:10A4C0008A68456012011A438461496881630262A7
:10A4D00030BD30B5026AFF2301339A430262026A3B
:10A4E0004568C3697024A3439C080B68A4002343F8
:10A4F00001246402A2438C68456024021443C361B2
:10A500004968C163046230BD30B5026A01231B0390
:10A510009A430262036A4568C26973242402A24313
:10A520000C68240214430122520393438A68456055
:10A5300012031A43C46149680164026230BD30B538
:10A54000036A046A6408640004628469F025AC4309
:10A55000120122430A24A3430B438261036230BDEC
:10A5600030B5036A1024A34303628469036A0F258C
:10A570002D031203AC432243A024A3430901194332
:10A580008261016230BD0000F0B50F4900220D4C20
:10A590000B461046A589643B10E00E5C771CFFB2A9
:10A5A0000F54BC46052E07D246009E5B5700DE5373
:10A5B00066468E54521C92B2401C80B2A842ECD324
:10A5C000A281F0BD40010020280C0020F8B501F068
:10A5D000F7F8284C0026A664207801250527ED030E
:10A5E0003F07030000F0BDFC04030B182C2E0122D2
:10A5F00029463846FDF727F8FFF778FC06E00122E8
:10A6000029463846FDF71FF8FBF730FF00222946A0
:10A610003846FDF718F815E0607B0122401C607396
:10A6200029463846FDF70FF8FCF706FA00222946BE
:10A630003846FDF708F8607B052803D9267001E04D
:10A64000FEF7C8FF02210C48FCF7F0FF00280FD0EE
:10A6500000200A49087001F0B3F80121084801F010
:10A66000B9FA002001F0E2FA002001F082FAF8BD08
:10A670000120EEE77000002000040050440200209A
:10A6800000D0232410B5818CC90707D001684A681F
:10A6900001235B049A43836A1A434A60818C8907C9
:10A6A00007D501684A6801231B049A43C36A1A4309
:10A6B0004A60818C490707D501684A6801239B04D9
:10A6C0009A43036B1A434A60818C090707D50168D6
:10A6D0004A680123DB039A43436B1A434A60818C27
:10A6E000C90607D50268916801231B039943836B50
:10A6F00019439160818C890607D501688A68012316
:10A700005B039A43C36B1A438A60818C490612D556
:10A7100003685A6801210905046C8A4322435A6080
:10A72000026C8A4207D10268516803235B05994392
:10A73000436C19435160818C090607D501684A684A
:10A740000123DB04806C9A4302434A6010BD000081
:10A75000F8B50446002680300660FCF77BFF05460E
:10A7600020680068124F000709D501212B460022FE
:10A7700049052046009700F0A1FA00280DD1206875
:10A78000006840070BD501212B4600228905204691
:10A79000009700F093FA002801D00320F8BD202094
:10A7A000A067E0672666603426750020F8BD0000CB
:10A7B000FFFFFF01F8B5154CC826E078002823D12B
:10A7C0006079002820D101206071114D686B00274D
:10A7D000002818D0686BC821081A0FE00D48E168FE
:10A7E000405C61698847E068401CE060E068C82818
:10A7F00000DBE760696BC820401A761EE168814281
:10A8000001D0002EEADC6771F8BD00005400002082
:10A81000000002407403002070B5224CE07800284C
:10A820003FD1207900283CD1012020711E4EF169D2
:10A8300000250906002933DA2156625791420AD1D0
:10A84000F06940062CD5A079002829D0A57120896F
:10A85000401C208124E0A179002903D1A0710A20A5
:10A8600000F04BFE00202056682148430F49421853
:10A87000206912181279B262401C00222061A2568F
:10A8800068235A43895881420ADC25612078401C9C
:10A8900020702078022800D12570A078401CA0707C
:10A8A000257170BD5400002000380140A402002032
:10A8B00010B5806A0022014640314A834A82FDF782
:10A8C000ABFF10BD70B5846AA06FE56F2168896821
:10A8D00000260906002906DA212804D15220065351
:10A8E000204600F06BF820688068400606D5222DCF
:10A8F00004D15A200653204600F047F82046803005
:10A9000001681022114301602046FDF785FF70BDEC
:10A9100010B501460968806A096889061CD40022BE
:10A920005A210A5201680A68FF2301339A430A60D8
:10A9300001688A68520852008A6001688A68402368
:10A940009A438A602021C167016E012904D1016800
:10A950000A6810239A430A60016E012902D0FEF7AB
:10A960003DF910BD5821095AFDF754FF10BD10B52F
:10A97000806A016E012902D0FEF731F910BD58211D
:10A98000095A4908FDF746FF10BD01680A68FF2310
:10A9900021339A430A6001688A68520852008A602B
:10A9A000016E012904D101680A6810239A430A60E4
:10A9B0002021C167002101664166704701680A686D
:10A9C000C0239A430A6020218167704770B5164CF6
:10A9D000E278002A0CD12279002A09D10122E27002
:10A9E0000025642903DC0222A256002A01DCE5705E
:10A9F00070BD0123E356682253430C4AD150012312
:10AA0000E356682673439B180A460146181DFAF759
:10AA1000C9FB6078401C60706078022800D16570C6
:10AA2000A078401EA070E2E754000020A40200209D
:10AA3000F8B50446016880682369E66918436369CC
:10AA4000002533431843724A0B68724E3340034368
:10AA50000B602168486803231B039843E36818438D
:10AA600048602168A069914201D0236A18438B682D
:10AA70000B263602B34303438B606749236867485C
:10AA80008B420CD1C0688007800F06D0012839D0D6
:10AA9000022835D0032821D11EE001271FE060499C
:10AAA0008B420AD1C0680C21084027D0042829D045
:10AAB000082825D00C2811D10EE093420ED1C16890
:10AAC00003208002014019D001208002091A19D008
:10AAD000091A15D0814201D1082700E010274F49FB
:10AAE000504840398600934232D1002F0CD0022FBB
:10AAF0000DD0042F10D0082F7FD126E00027EEE7DD
:10AB00000227ECE70427EAE7FDF7A8F906E0096861
:10AB1000C90605D4304603E0FDF7C0F9002872D01D
:10AB2000626851005118814267D81103814264D391
:10AB3000010E06025008002330185941FAF702FBB3
:10AB400003210902411A384A55E00120C003E7E712
:10AB50000122E369D20393422BD13B0000F001FABA
:10AB60000906090C4D114D4D4D274D00FDF776F9A5
:10AB700009E0FDF783F906E00968C90605D4304607
:10AB800003E0FDF78BF900283DD0616840004A08DA
:10AB90008018FAF7ADFA80B20146244A1039914282
:10ABA0002BD8511C01400007400F084329E01046F4
:10ABB000EBE73B0000F0D5F90906090C2112212131
:10ABC00021232100FDF74AF90AE0FDF757F907E0D4
:10ABD0000968C90606D4304604E00EE0FDF75EF9C8
:10ABE000002810D061684A081018FAF781FA80B27C
:10ABF00001460E4A1039914203D9012503E010465F
:10AC0000F0E72168C86000206066A0662846F8BDAD
:10AC100000480040F369FFEF003801404010024057
:10AC20000044004000093D00FFFC0F00EFFF000062
:10AC3000F8B5044641654030002627460283803738
:10AC40003E602220E0672546206F603500281CD03A
:10AC50001749C162216F17480863216F164848637E
:10AC6000206F8663236F606D9C4613462168024601
:10AC700060462431FCF72EFB002806D010203860F7
:10AC80002E752020A0670120F8BD2E752068016870
:10AC9000FF220132114301602068816801221143C3
:10ACA0008160206881684022114381600020F8BDE6
:10ACB00011A900086FA90008C5A80008FFB581B058
:10ACC00005460F46044660350A9E39E0701C37D0B1
:10ACD000FCF7C0FC0499401AB04222D8002E20D0C4
:10ACE0002068016849072BD5C069C043000527D4F7
:10ACF00001202168C002086220680168FF22A13299
:10AD000091430160206881684908490081602020E2
:10AD1000A067E0678034206000202875032005B01C
:10AD2000F0BD20680168FF22A132914301602068D4
:10AD300081684908490081602020A067E067EBE74F
:10AD40002068C1693846884305D0002103988142B4
:10AD5000BCD00020E3E70121F8E7000010B504496A
:10AD60001020096808620248FDF758FD10BD000078
:10AD7000DC11002001B501231A4669460248FDF79F
:10AD80002FFF0248C06908BDDC11002000380140D7
:10AD900070B50D460646002403E0305DFFF7EAFF7C
:10ADA000641CAC42F9DB70BD01490120887070471A
:10ADB0005400002010B5FEF7B9FAFEF7E3FBC822F5
:10ADC00002490348FDF7DAFE10BD000074030020BD
:10ADD000DC110020F8B53E4C002321783D4A1D4689
:10ADE000082910D0072947D0062950D0052952D06C
:10ADF000042953D0032954D0002956D0012958D012
:10AE000002295AD05BE0A17800264A1F04E0314FA6
:10AE1000BF5DFB189BB2761C9642F8DB66792779FA
:10AE20009A195118E3786278C9188918C919401815
:10AE3000C0430006000E1AD1012E14D0022E16D1E6
:10AE400025482449C018FAF7ADF901F093FC6420B5
:10AE500000F04CFBBFF34F8F21492048C860BFF37F
:10AE60004F8F00BFFDE759081046FFF775F92570B1
:10AE7000E570A570A571F8BDA1795054491CC8B200
:10AE8000A071A178491F8842F5D1082001E06070C7
:10AE900007202070F8BDE0700620FAE760710520F9
:10AEA000F7E7A070E5700420F3E7552807D10120EB
:10AEB000EFE7AA2803D10220EBE7032803D025708F
:10AEC000E570A570F8BD032020702071F8BD00006A
:10AED00038010020560900203C0400200400FA0537
:10AEE00000ED00E00FB410B503A9044B044A02982A
:10AEF00000F0AAF910BC08BC04B018476DBE0008E9
:10AF0000600200202021020C01D010211046020A0C
:10AF100001D010460839020901D01046091F8208E5
:10AF200001D01046891E420801D0881E7047081AB9
:10AF30007047F8B5040C8BB2264682B25E430D0C06
:10AF40001046370C584336048019002179411646C3
:10AF50006E43370C36048019794126466E438919B1
:10AF6000F8BD30B47446641E2578641CAB4200D230
:10AF70001D46635D5B00E31830BC18478307FF2262
:10AF8000DB0E9A408907090E9940002808DB8308E8
:10AF900009489B001B1818689043084318607047C5
:10AFA0000007000F0838830804489B001B18D86965
:10AFB00090430843D861704700E400E000ED00E0F2
:10AFC000BFF34F8F04490348C860BFF34F8F00BFE2
:10AFD000FDE700000400FA0500ED00E0F8B50446C6
:10AFE0004F1EC8000838211815461E4608684968D3
:10AFF0003A4606239A4310D02A463346FAF74CFACB
:10B000003A46D200083AA3181A687F1E5B68FAF71E
:10B0100091F906223B469343EED1022F23D0042F11
:10B0200011D0062F2FD12A463346FAF735FAE36AB4
:10B03000A26AFAF77FF92A463346FAF72DFA636ACD
:10B04000226AFAF777F92A463346FAF725FAE369CE
:10B05000A269FAF76FF92A463346FAF71DFA6369CF
:10B060002269FAF767F92A463346FAF715FAE368D0
:10B07000A268FAF75FF92A463346FAF70DFA6368D1
:10B080002268FAF757F9F8BD002210B513461046AA
:10B090000149FAF769FA10BD0000F03F10B501222E
:10B0A000FAF7DAFA10BD002210B513461046114621
:10B0B000FAF75AFA10BD02E008C8121F08C1002AA8
:10B0C000FAD170477047002001E001C1121F002A29
:10B0D000FBD17047014908607047000064020020FE
:10B0E00038B504466D20694608706B460122074951
:10B0F0002E2000F04FFE0649002C01D0054A00E04A
:10B10000054A2E2000F02CFE38BD00000608000085
:10B1100006180000070600000716000038B50446B0
:10B120006B4602220021362000F0EEFCB321230002
:10B13000FFF717FF0E0F08153A3A3A3A1C273A3A2A
:10B140002F34483A00216846017040784108490090
:10B1500014E06946087880088000401C04E06946D5
:10B16000087880088000801C08701DE0684602781E
:10B170000A4048320270417880200143684641709D
:10B1800012E0684602780A40027040784106490E93
:10B19000F4E7694648780221084303E069464878A5
:10B1A000FD210840694648706B4601220021362087
:10B1B00000F0F0FD012200AB11463620013300F013
:10B1C000E9FD38BD69460878CF210840694620303E
:10B1D000CAE708B5032168464170012101706B463A
:10B1E00002220021362000F0D5FD0122D2030621E3
:10B1F0002D2000F0B5FD012000F078F90120FFF7C7
:10B200008DFF08BD08B5020A69464A7008706B4692
:10B21000022204212D2000F0BDFD032069460870A4
:10B220006B46012206212D2000F0B4FD0020694666
:10B2300008706B46012206212D2000F0ABFD0A218B
:10B240002D2000F00FFC08BDFFB58DB00446002591
:10B2500006E025280AD0109A0F999047641C6D1CAF
:10B2600020780028F5D1284611B0F0BD0027012133
:10B27000484A009700E00743641C23780846203BB7
:10B2800098401042F7D120782E2817D10420074388
:10B290006078641C2A280CD10E98641C02C80091A6
:10B2A0000E900BE000990A22514330394018641C7B
:10B2B00000902078014630390929F3D920780028F8
:10B2C000D1D0642808D0692806D075281ED0109ADD
:10B2D0000F9990476D1C5BE00A200E99019001C9FF
:10B2E0000E91002802DA40422D2102E0390504D5F2
:10B2F0002B216A461172012103E0F90704D02021B5
:10B30000F7E70BAE0B910DE00021FAE70A200E994A
:10B31000019001C90E91F7E70199F9F7E9FE303183
:10B32000761E31700028F7D103A8801B20300190D1
:10B33000780701D5009801E001200090019988422A
:10B3400001DD401A00E000200027009006E002A87E
:10B35000109AC05D0F9990476D1C7F1C0B98874217
:10B36000F5DB04E0109A30200F9990476D1C00998E
:10B37000481E00900029F5DC05E03078109A761C14
:10B380000F9990476D1C0199481E01900029F4DC2B
:10B39000641C65E709280100F3B585B0069D00220D
:10B3A0006D1E39E00121069B8C4600219B1A5B1E15
:10B3B0002CE08C000659271803977F68BE46764517
:10B3C00023DD0027BC460296154F4E00BF5B019758
:10B3D000134F64377F5C049777460751104C104F2A
:10B3E000341900946488BC533C4664346418A646FF
:10B3F00066783C4664346654039E029C7460009CEC
:10B40000019F67807446049F6770491C8B42D0DCA3
:10B410006146002902D1521CAA42C3DB07B0F0BD2D
:10B42000C40B0020F8B54A002B4B520DD6182B4AFE
:10B430000C460546142E2BDA002E12DA284BF9F7AB
:10B4400079FF00221346FAF70DFA40D2002C03DAF6
:10B450000124E40700253AE02046284337D0214C58
:10B4600014E0214F0B46F7403B402B4331D01C4B9F
:10B47000F9F760FF00221346FAF7F4F927D2002CFF
:10B4800003DD01200005F0400419BC4300251EE047
:10B49000332E1EDC33460027143BFF43DF40384287
:10B4A00017D00F4BF9F7F0FF00221346FAF7DAF93D
:10B4B0000DD2002C0ADD142E0CD03420811B01206B
:10B4C00088404019A84200D2641C0546BD4321466D
:10B4D0002846F8BD641CF9E701FCFFFF9C75008855
:10B4E0003CE4377E0000F03FFFFF0F007D2110B5E8
:10B4F000C900484300F001F810BD002140E000BF42
:10B5000000BF00BF00BF00BF00BF00BF00BF00BF43
:10B5100000BF00BF00BF00BF00BF00BF00BF00BF33
:10B5200000BF00BF00BF00BF00BF00BF00BF00BF23
:10B5300000BF00BF00BF00BF00BF00BF00BF00BF13
:10B5400000BF00BF00BF00BF00BF00BF00BF00BF03
:10B5500000BF00BF00BF00BF00BF00BF00BF00BFF3
:10B5600000BF00BF00BF00BF00BF00BF00BF00BFE3
:10B5700000BF00BF00BF00BF00BF00BF00BF491C2D
:10B580008142BCD370470000FEB504460020019004
:10B5900000906079734940000E5A61782578491E01
:10B5A0007148CFB20163042D77D0072D75D00021EB
:10B5B0000291217801736C49E3790122920589692E
:10B5C000002B6CD0914381616748217A4173217AC5
:10B5D00082698907890B0A4382610021042000F0F7
:10B5E000CAFB324661492E2000F0BAFB3846FFF70D
:10B5F00077FD5F4E0522705D810040185D4943185C
:10B6000007212B2000F0C6FB5B49029801220B1892
:10B610000B21282000F0BEFB705D584980000A58BD
:10B620000C21282000F0A7FBE07955498000401844
:10B63000A1794900425A0221272000F091FB51488C
:10B640007E00825B0421272000F08AFBE07900283D
:10B6500029D0A07804282CD02820694608722022FE
:10B660000621272000F07CFB02AB012226212720A7
:10B6700000F090FB444938014018E17889004258B5
:10B680000821272000F077FBA17A601C627A09026A
:10B69000114313D016E000E001E0012188E71143D7
:10B6A000F608816190E764220621272000F058FB0C
:10B6B000E0E71020694608720246D1E7334901727B
:10B6C000090A4172417A007A0A02024320212720A6
:10B6D00000F046FB2E4F0C2123203A6800F04BFB74
:10B6E000F01982880421232000F03AFBA079002879
:10B6F0000BD0E0792749012243180021212000F0D6
:10B7000049FB03200190012000902A07120F10012D
:10B710000243607800218007000B02430198000576
:10B7200002430098400402432079C00640090243C6
:10B730006079C00602431F2000F01DFBA0786178ED
:10B740000123084302040848DB030261E17949034D
:10B7500019430A4302610021082000F00CFB00207D
:10B76000FEBD000048C80008680200200428000050
:10B77000F0C700082400002042000020F8C700089D
:10B7800018C8000824C8000828C800084110000094
:10B7900010C800084400002010B5044604213620DB
:10B7A00000F060F90121C902002C01D0084300E03B
:10B7B000884302460421362000F0DDFA10BD000067
:10B7C00038B540206946087000210E2000F04AF983
:10B7D0000446002211460E2000F0CDFA6B460122ED
:10B7E00000210D2000F0D6FA074A00210F2000F0BA
:10B7F000C2FA00F09BFA224600210E2000F0BBFAAC
:10B8000002480021017338BDF8FF27248802002078
:10B8100070B50546164600240846F9F7FBFF0222DC
:10B82000F9F71AFFF9F78CFFFF2800DDFF20264902
:10B830000A46083A012E09D0042D27D0072D25D01D
:10B84000515D1A225143214A89182EE0042D08D057
:10B85000072D06D0515D252251431B4A0832891815
:10B860000EE0495D44225143184A883A891800E0A5
:10B87000641C0A5D8242FBDB20461C381AE0641C13
:10B880000A5D8242FBDB2046173813E0495D3B220C
:10B8900051430E4A6832891800E0641C0A5D8242F6
:10B8A000FBDB20461E3805E0641C0A5D8242FBDBA0
:10B8B00020461138F9F7E6FEF9F7ACFF044A054BCC
:10B8C000F9F7EAFD70BD000082C80008A6C90008AB
:10B8D0007B14AE47E17A843FFEB5054604206946F5
:10B8E0000870514C0020607521462031206348715A
:10B8F0000873A0836063A06300F0E2F84B4E206001
:10B9000002E000F0DDF82060B042FAD10020FFF73D
:10B9100005FC00F0D5F8464E20603078242801D987
:10B92000243806E00621F9F7E3FB0622101A40014D
:10B930000843020601040A4301020A430243B260BB
:10B94000706000211E2000F016FA00F0B9F82060A7
:10B950006B4601220021242000F01CFA1E20FFF774
:10B9600051FC86B2300AA0730420FFF74BFC074657
:10B9700000F0A6F820603806000E0DD002206946BF
:10B98000087101AB012212212D2000F003FAA08BD7
:10B99000012109030843A08300F092F820600620EB
:10B9A000FFF730FC60600720FFF72CFCA060F0067A
:10B9B000C00E207501D110202075C0B200F026FA0B
:10B9C000E80707D0FFF705FCA08B0121C902084357
:10B9D000A0830AE00521362000F02EF81549084022
:10B9E00002460521362000F0BBF90120FFF796FB47
:10B9F0000021042000F036F8A0610021262000F08C
:10BA000031F815218903084302460021262000F061
:10BA1000B2F900222621362000F0A2F900F050F8F9
:10BA200020600020FEBD0000680200203001CADE58
:10BA300018000020FFFD000038B5094C89B280B223
:10BA40006B46022200F060F8002806D16846407874
:10BA5000010268460078081884B2204638BD00000C
:10BA6000FFFF000038B50024E44389B280B26B4682
:10BA7000042200F049F8002806D103216846435CFF
:10BA80002202D418491EFAD5204638BD38B5002404
:10BA90006B4603222821272000F036F80220694651
:10BAA0000B5C2202D418401EFAD5E00202D50348EE
:10BAB000204338BDE002C00A38BD00000000F0FF9E
:10BAC00010B500210846FFF7CDFF10BD10B50446A4
:10BAD00005211520FFF7B0FFE08100212E20FFF7A0
:10BAE000ABFF2080231D08220021122000F00CF85B
:10BAF00007211520FFF7A0FF608000211020FFF72D
:10BB0000B1FF000DA08110BD38B5002909D0402437
:10BB100020436C462070C8B27F2906D8607002208E
:10BB20000AE069460870012006E0802420436C4644
:10BB30006070C809A0700320694600F0A7FD38BDF9
:10BB400010B5144603460A4621461120FFF7DCFFD4
:10BB500010BD10B50346052200211520FFF7D4FFC4
:10BB600010BD10B50346052200211720FFF7CCFFBA
:10BB700010BD38B5054600206946087000F0D6F8BB
:10BB8000FF2401342246002D01D00322120200219D
:10BB90000D2000F0E5F8002D13D06B4601220321A3
:10BBA0000F20FFF7B1FF68460078000709D5FFF7BF
:10BBB00007FE224600210D2000F0D2F80020C043ED
:10BBC00038BD002038BD10B5024601210A2000F022
:10BBD000D2F810BD70B50D46044600210E20FFF7C7
:10BBE00041FF002D01D0204300E0A0430246002188
:10BBF0000E2000F0C0F870BD10B5044600211A20D8
:10BC0000FFF730FF000D22030005120B0243002155
:10BC10001A2000F0B0F810BD10B5024602492E20DF
:10BC200000F09EF810BD000004180000F8B50546AD
:10BC30006B46012203210420FFF766FF0126114C09
:10BC40003607002D0DD02A4600210C2000F088F880
:10BC5000694608781021084369460870A069304396
:10BC600007E069460878EF21084069460870A06936
:10BC7000B0430B46A06101220321042000F08AF8A2
:10BC8000F8BD00006802002010B50246002118200F
:10BC900000F066F810BD0000F8B5074600256846BC
:10BCA0000570B807204C2E4600280ADA8020694625
:10BCB00008706B46012200210D2000F06BF8012076
:10BCC0002073F8076946087821D0062108436946A1
:10BCD00008706B46012200210D2000F05BF8032163
:10BCE0000F20FFF7A9FE8121C900084219D040208A
:10BCF000694608706B46012200210D2000F04AF8C9
:10BD00000020FFF749FD00252673ED4309E00221DD
:10BD10000843694608706B46012200210D2000F09F
:10BD200039F82846F8BD0000880200201CB56B4693
:10BD3000012203210F20FFF7E7FE6846007840222A
:10BD4000C1091040C9014000814208D00120694664
:10BD50000871024601AB03210D2000F01BF81CBD49
:10BD600008B56B461A70120A5A7089B280B2022264
:10BD700000F010F808BD38B500236C46E254120AF2
:10BD80005B1C042BFADB89B280B22346042200F04C
:10BD900001F838BD38B58024002909D0C0252843D2
:10BDA0006D462870C8B27F2907D86870022009E064
:10BDB000204369460870012004E020436870C809E8
:10BDC000A8700320694600F0EFFC38BD10B514469A
:10BDD000012312189B029A4202D90020C04310BDD1
:10BDE0000B46821E21460920FFF7D4FF002010BD1C
:10BDF00010B5054A8905126901430A43002108204C
:10BE0000FFF7B9FF002010BD6802002038B50446D6
:10BE10006B4601220E212B20FFF776FE6846007844
:10BE2000E10640094001C90E0143684601706B46B6
:10BE300001220E212B20FFF7ADFF38BD10B50022E7
:10BE40000A60835CD400A3400C68521C1B190B6071
:10BE5000042AF6DB10BD10B5002142541C06120A5C
:10BE600022431B0A491C0429F7DB10BD13B501232B
:10BE70001A4669460248FCF7B3FE00981CBD000054
:10BE8000DC1100207CB5002425466846FFF761FEE2
:10BE900004206946220E2D02154322020C5C144335
:10BEA000401EF7D5204629467CBD7CB5002425469A
:10BEB0006846FFF74EFE04206946220E2D02154308
:10BEC00022020C5C1443401EF7D5204629467CBD57
:10BED0007CB5002425466846FFF743FE04206946EA
:10BEE000220E2D02154322020C5C1443401EF7D58E
:10BEF000204629467CBD0000F0B5C54A00248FB01D
:10BF000091420ADA4B005B08934206D801254A00A9
:10BF10006D05EA4205D1002803D0FFF7BFF80FB046
:10BF2000F0BD01252D05A94219DA034308D00029E7
:10BF300010DA0120FFF7CEF8FFF7B5F80FB0F0BD2B
:10BF40000220FFF7C7F8FFF79FF80122D207514000
:10BF50000FB0F0BD3524E4433622F9F77DFB0A1516
:10BF6000AC4B1219D4180A03120BAB49AB4B561841
:10BF70002E403146594011430192321512190B924D
:10BF80000022F9F77BFA019A0446921C1003A44E92
:10BF9000000B0D467E44032860D220467368326849
:10BFA000F9F74CFC1CD10B98002815D0F9F77CFB55
:10BFB00004460E469B4A9C4BF9F76EFA0D4607461F
:10BFC0009A4A9B4B20463146F9F766FA3A462B4689
:10BFD000F9F7B0F90FB0F0BD716830680FB0F0BD7F
:10BFE000944A954B20462946F9F756FA0022934B7E
:10BFF000F9F74AFA06460F4622462B4610461946DE
:10C00000F9F74AFA32463B46F9F746FA06460B98E4
:10C010000F4600281DD0F9F747FB824A824B059155
:10C020000490F9F739FA32463B46F9F72DFA2246E1
:10C030002B46F9F723FA04460D467C4A7C4B0599BA
:10C040000498F9F729FA22462B46F9F717FA0FB0A8
:10C05000F0BD0B46324620462946C4E001230022AB
:10C060009B072046F9F766F902460B46204629460B
:10C07000F9F77AFA06460F460B98F9F715FB3246A0
:10C080003B460591049010461946F9F705FA0991C7
:10C090000C906B490198099B421800920C9A194622
:10C0A0001046F9F7F9F9024607910A906549019897
:10C0B0000B1A6548019303217844079BFEF78EFF16
:10C0C000079B0A9AF9F7E8F90E905F480D91042151
:10C0D0007844079B0A9AFEF781FF099B0C9AF9F7AF
:10C0E000DBF9019B009A1A4300920D9B0E9AF9F717
:10C0F00021F9009A01910C90002A4DDD0022D243D3
:10C1000020462946F9F7A8FA22462B46F9F7C4F942
:10C1100000910A900B9800282BD0424A424B059977
:10C120000498F9F7B9F907910E90019B0C9A0099C0
:10C130000A98F9F7FFF832463B46F9F7ADF9079B45
:10C140000E9AF9F7F7F8009B0A9AF9F79DF922463B
:10C150002B46F9F793F904460D46344A344B0599BA
:10C160000498F9F799F922462B46F9F787F90FB0A9
:10C17000F0BD019B0C9A0A98F9F7DCF832463B4671
:10C18000F9F78AF9009B0A9AF9F77EF922462B46BD
:10C19000F9F77AF90FB0F0BD0B98002827D0214AA3
:10C1A000214B05990498F9F777F9079100902046FB
:10C1B0002946019B0C9AF9F761F932463B46F9F79B
:10C1C0006BF9079B009AF9F759F922462B46F9F7C4
:10C1D00055F904460D46154A154B05990498F9F78B
:10C1E0005BF922462B46F9F749F90FB0F0BD0B4633
:10C1F000204629460C9AF9F741F932463B46F9F7B1
:10C200004BF922462B46F9F73FF90FB0F0BD00007D
:10C210000000F07F01FCFFFF645F09000000F03FB9
:10C22000480B0000763C7935EF39EA3D0000E0FE2E
:10C23000422EE63F555555555555D53F0000E03F38
:10C2400086EBF9FF51B80600EC090000F8B504468A
:10C250003048002581420ADA4A005208824206D854
:10C26000012348005B05D84205D1002C03D02046AD
:10C27000FEF714FFF8BD01231B05994219DA22438A
:10C2800007D000290EDA0120FEF724FFFEF70BFF8E
:10C29000F8BD0220FEF71EFFFEF7F6FE0122D207D0
:10C2A0005140F8BD3525ED4336222046F9F7D4F943
:10C2B000044608154019184A0D038018C20F174983
:10C2C0002D0B891A09050D438018F9F7EDF906467B
:10C2D0000F4620462946FFF70FFE114A114BF9F78A
:10C2E000DBF804460D46104A104B30463946F9F744
:10C2F000D3F822462B46F9F71DF80D4604460C4AA2
:10C300000C4B30463946F9F7C7F822462B46F9F769
:10C3100011F8F8BD0000F07F01FCFFFFFF030000F3
:10C320000EE526157BCBDB3F362BF111F3FE593D95
:10C3300000609F501344D33FFBF79AF9FDF7D6FFF7
:10C34000FDF708F836493748002522C005608561A9
:10C35000C56135490562C1600838FBF72DFBFCF764
:10C36000E5FFFDF70FF9FDF7ABF8FCF7ABFFFDF7C5
:10C37000C9F8052401222407D1032046FBF763F9FD
:10C38000FDF724FDF9F73CFCFAF7F4F9FAF7C2F9E6
:10C3900001212648FFF71EFC0020FFF747FC002084
:10C3A000FFF7E7FB0122170339462046FBF74BF95D
:10C3B0001C48C8221E49C830FCF7E0FB1D4C1E4833
:10C3C0001E4EE572E27A8254521CD1B2E172FF290C
:10C3D000F8D3A079002820D0A571657272B62078B4
:10C3E0000F2804D9B761FEF7F1F8B7620CE001221B
:10C3F00051033046FBF727F9FEF7E8F80121002248
:10C4000049033046FBF71FF962B6FCF765FD208D46
:10C410000028DED0401E2085DBE7FCF75DFDD8E775
:10C42000007C004014110020FFFF000000D02324F6
:10C4300074030020080200208C0F0020000400502C
:10C4400010B50446FCF7E4FC4E20FCF7B4FCFCF706
:10C4500018FDE0B2FCF7AFFCFCF713FDFCF7D8FCCD
:10C460004F20FCF7A8FCFCF70CFD0020FCF776FC45
:10C470000446FCF7E8FC204610BD70B50D460446A6
:10C48000FCF7C6FC4E20FCF796FCFCF7FAFCE0B289
:10C49000FCF791FCFCF7F5FC2846FCF78CFCFCF75C
:10C4A000F0FCFCF7D0FC0A20FFF727F870BD000075
:10C4B00010B52421002000F04DF81B48FFF71DF8AF
:10C4C00000210F2000F046F80521102000F042F86E
:10C4D0000421112000F03EF883217F2000F03AF87B
:10C4E00069217F2000F036F8BD217F2000F032F86E
:10C4F0000E480078262804D1002240218C2000F02C
:10C5000019F8012000F02AF8094814210187282091
:10C5100000F020F80A20FEF7F0FF012000F036F8C6
:10C52000012000F043F810BD204E00000000002064
:10C530003C040020F8B517460E4605460024FFF7D8
:10C540007FFF3946B44331402143284600F002F8CA
:10C550000020F8BD10B5FFF790FF10BD10B5002802
:10C560000AD000212720FFF7F5FF04211920FFF74B
:10C57000F1FF8721162005E000211620FFF7EAFFD2
:10C5800000211920FFF7E6FF10BD000010B50028BC
:10C5900001D0002200E0802280211120FFF7CAFF95
:10C5A0000148FEF7AAFF10BDA086010010B50028C3
:10C5B00011D001212F20FFF7CDFF62213020FFF79E
:10C5C000C9FF46213120FFF7C5FF32210846FFF79A
:10C5D000C1FFA22100E022213320FFF7BBFF10BDE5
:10C5E0000C480D4A0188914210D1C18832290DD3DF
:10C5F000C18E43290AD8818F012907D8C08F01280D
:10C6000004D8044840308088012801D901207047AF
:10C61000002070473C040020AA55000010B5C82235
:10C6200016491748FAF72EF91448164902888A4223
:10C6300023D0018014498180FF21F531C1800A2176
:10C64000018100211E224181D24382810122C281C7
:10C6500081834323C386022303877823438782870A
:10C66000C28702464032118451849184C1839180F3
:10C6700014238382118200F07DF810BD3C04002059
:10C6800000FC0008AA55000034120000F0B58C46EA
:10C6900000251026052109078E620E4C08E067462A
:10C6A0007F5DE760A768FF07FCD0E7681F706D1C1F
:10C6B0008542F4DB0020074606E0E760A568ED0749
:10C6C000FCD0E5681D54401C9042F6D38E610020DA
:10C6D000F0BD000000300140F0B513B406460199EA
:10C6E000F9F7CEF904460D4602460B46304601994D
:10C6F000F8F7C4FE064601981B4B0F4600280CDADB
:10C7000000223046F9F79AF80CD90022174B304630
:10C710003946F9F7A7F81DD214E000223046F9F7A0
:10C720008DF808D20022124B20462946F8F7A6FEC3
:10C7300004460D460EE000220C4B30463946F9F710
:10C7400091F807D800220A4B20462946F8F7F2FD57
:10C7500004460D46019A69004908D20FD2072046C7
:10C76000114303B0F0BD00000000E0BF0000E03F57
:10C770000000F03F10B5FFF733FF002801D0012083
:10C7800010BD72B6C821064C2046FAF761F80028A1
:10C7900004D0C82203492046FAF7FEF862B610BD5D
:10C7A00000FC00083C040020F0B5002510260527F9
:10C7B0009C463F070B46BE620C4C06E0595DE160AB
:10C7C000A168C907FCD0E1686D1C8542F6DB00203A
:10C7D00007E06146095CE160A168C907FCD0E16837
:10C7E000401C9042F5D3BE610020F0BD00300140F6
:10C7F0000000010203040005405C0000A05C04008E
:10C80000C06C0800805C0400E03F1E00E07D1E005C
:10C8100007A9022570889B880A00160001000600FF
:10C820000100020087008D002D001A3152001A33DA
:10C830009A001A351D011A376B003B31BE003B339D
:10C840005E013B3596023B37000099599959EB51EF
:10C850008F421E45142E0080EB51F5283333E13A08
:10C86000703DE13AC235852BC2353333C235C2350E
:10C87000AE47E13A5138A3305138000001020003BD
:10C88000000000000000000000010103040507098A
:10C890000B0C0D0F121417191C1E2124282B2F32DC
:10C8A000363A3F42474C5259626D7F9BDEFFFF0193
:10C8B0000204050608090A0C0D0F121416181B1D98
:10C8C000202326292C2F33373A3E42474E55606F9E
:10C8D00087C2F0FF01020304050708090A0C0E10C5
:10C8E000121416181A1C1F2124272A2D3134373B05
:10C8F0003F454C556278ADD5FF01010203040506A2
:10C90000060708090B0C0E0F1012141517191B1D22
:10C910001F222426292C30353B44537894FF0707E7
:10C920000809090A0B0B0C0D0E0F10111213141528
:10C930001617181A1B1C1E1F20222426282A2C2EEC
:10C9400030323437393B3D3F4244474A4E515559C6
:10C950005E63686E747B828B96A4B6CFEEFFFFFF9A
:10C96000FFFF0405050506060707070809090A0A67
:10C970000B0B0C0D0D0E0F101111121314151617B1
:10C98000191A1B1D1E1F202223242627282A2C2E7D
:10C99000303234373A3D4044484B50555C65707FE7
:10C9A00093A8B6C2CDFF010202030405070A0D10C9
:10C9B0001316181B1E2023262B30384E65789DFF3A
:10C9C00001020203040406090C0E111315181A1CA7
:10C9D0001F21252A314459698AFF010102030304FA
:10C9E00005080A0D0F11131517191B1E21252C3CC4
:10C9F0004F5D7AFF010101020203040607090A0CD8
:10CA00000D0F10111315171A1E2A374155FF07086D
:10CA10000809090A0B0C0D0D0E0F1010111213133B
:10CA200014151618191B1C1D1E2021222325272929
:10CA30002B2D303235383C40444A5159626D7A884A
:10CA4000929AA2B2DCF9FFFFFF040505050606076E
:10CA500007080809090A0A0A0B0B0C0D0D0E0F1026
:10CA600010111213131415161718191A1C1D1F2153
:10CA70002325272A2E32363C434B535A5F646E8758
:10CA800099ACC0FF00000000000000000102030498
:10CA900006070809030406080C10182030000000DF
:10CAA000000102030400000004FA97999999D93F04
:10CAB000AF788E1DC571CC3F9FC678D0099AC33F11
:10CAC000935555555555E53F599322942449D23FE6
:10CAD000DE03CB966446C73F44523EDF12F1C23FAD
:10CAE000000000000000000008CB0008000000204B
:10CAF00068020000205B000850CB0008680200209C
:10CB000068150000C6B00008022327130704380D7B
:10CB1000091E080540082609104008560A131D047E
:10CB20003B08BE0516D8BC4010085201033AC84263
:10CB3000079852030CE5800C14020214B70909018E
:10CB400002038149F501FFC134803F019204922024
:04000005080050C1DE
:00000001FF
